:1000000000400020E53E0000253F0000273F0000A3
:1000100000000000000000000000000000000000E0
:10002000000000000000000000000000293F000068
:1000300000000000000000002B3F00002D3F0000EA
:100040002F3F00002F3F0000194700002F3F000006
:100050002F3F0000000000002F3F00002F3F000056
:100060002F3F00005D4100002F3F00002F3F0000A8
:100070002F3F00002F3F00002F3F00002F3F0000C8
:100080002F3F0000BD4700002F3F00002F3F000022
:100090002F3F00002F3F00002F3F00002F3F0000A8
:1000A0002F3F00002F3F0000000000000000000074
:1000B0000000000000000000000000000000000040
:1000C000054B0648033310B51B1A062B03D9044B06
:1000D000002B00D0984710BDD4000020D400002091
:1000E000000000000648074910B5091A8910CB0F17
:1000F0005918491003D0044B002B00D0984710BD6D
:10010000D4000020D40000200000000010B5074CEF
:100110002378002B09D1FFF7D3FF054B002B02D02A
:10012000044800E000BF0123237010BDD40000206C
:10013000000000009C6C0000094B10B5002B03D0A0
:100140000849094800E000BF08480368002B02D1B5
:10015000FFF7C8FF10BD064B002BF9D09847F7E713
:1001600000000000D80000209C6C0000D00000209F
:1001700000000000164B002B00D1144B9D4640227E
:1001800092029A1A924600218B460F461348144A4F
:10019000121A04F08CFD0F4B002B00D098470E4B29
:1001A000002B00D098470020002104000D000D48CE
:1001B000002802D00C4800E000BF04F035FD20000C
:1001C000290004F0C1FA04F009FDC046000008004F
:1001D000004000200000000000000000D4000020CB
:1001E000EC1E00200000000000000000012303407E
:1001F0000200181E04D1042A03D91068000900E087
:100200000020704710B50400FFF7F0FF0300012045
:10021000002B0BD0013B9B00181DE2181279002A1D
:1002200003D001338342F8D100E0180010BD012251
:10023000016810B5114201D0002903DA102001F045
:10024000ABFD03E04910062001F05EFE10BD016821
:1002500010B5CB0701D5002903DA102001F09CFD71
:1002600006E04910033189100022052001F04CFE00
:1002700010BD70B50568AB0728D1042D26D90F2312
:100280002A6846681340062B09D12800FFF7AEFF05
:10029000012383421DDC9A00AE500133F9E7052BA0
:1002A00014D1F30703D4132001F076FD12E0761089
:1002B000FF2EF8D82800FFF799FF2C1D230080009F
:1002C0002018984205D91E700133FAE70B2001F07F
:1002D00063FD002070BD70B50468E30701D41120F0
:1002E0002DE04568AB0729D1042D27D90F262B68AF
:1002F00064101E40062E0BD1002C04DD2800FFF7F1
:1003000075FF844201DD122019E0A400605918E055
:10031000331F012B12D82800FFF768FF8000042E3E
:1003200002D12800FFF76EFF002CECDDA042EADBD3
:1003300001232C19E0784000184302E00B2001F063
:100340002BFD70BDF8B5012304681C4201D11120BA
:100350002FE00325466835402AD1042E28D90F23E3
:100360003268641087681340062B0BD1002C04DD23
:100370003000FFF73BFF844201DD122019E0A400AA
:10038000A75113E0052B13D1002CF6DD3000FFF749
:100390002DFF80008442F0DC01231F4201D1132095
:1003A00007E07F10FF2FFAD83419E770280002E029
:1003B0000B2001F0F1FCF8BD006810B5830717D1E0
:1003C000042815D90F2302681340062B02D1FFF72A
:1003D0000DFF0BE0052B05D1FFF708FFC00001233F
:1003E000184308E0042B03D1FFF70CFF4000F6E7A9
:1003F0000B2001F0D1FC10BD10B5032400680440AF
:1004000006D1042804D90F2302681340042B01D01D
:100410000E200CE001F0B4FD1022210005F004F9DB
:1004200080239B05C218054B9A4203D9142001F082
:10043000B3FC02E001234000184310BDFFFFFF3F63
:1004400010B501240368234202D04268224203D13E
:100450000D2001F0A1FC08E004495B1052101B07BD
:100460000A40134318684000204310BDFCFFFF0FF3
:100470000121036810B50B4205D042680A4202D040
:100480008068084203D10D2001F086FC08E0054990
:100490005B1052101B070A404010134318600020E5
:1004A00010BDC046FCFFFF0F012303400200181ED1
:1004B00001D0501002E00D22014B1A707047C04667
:1004C000F0000020012303400200181E04D1042A7A
:1004D00003D91068000900E00020704770B50D00D6
:1004E0000400FFF7EFFF86002800FFF7EBFF830013
:1004F00000209E420ED1231D9E1904351A009E42F3
:1005000007D929781278013301358A42F6D00020C4
:1005100000E0012070BD0000F0B585B003930190AC
:1005200002912D4E2D4B002A02D002223270013A48
:1005300000251A601B68F554019B9D424ADA029A15
:10054000AB00D058254B1C68C8239B0037191C1BD7
:100550000123184202D04310214A1FE0214A0028FB
:1005600002D0042805D1204A2100380004F066FF9B
:1005700018E0042810D90F2302681340042B04D17B
:1005800001F0FEFC194A030008E0062B05D1FFF735
:1005900099FF174A030001E00123164A21003800A1
:1005A00004F04CFF300004F0A5FF039B0B4A002B26
:1005B00001D110600CE0019B013B9D42F9DA0E4B2A
:1005C0009842F6DC431C1360202232540022F2547D
:1005D0000135B1E705B0F0BDFC000020F8000020B7
:1005E000F5630000C8630000CE63000014660000DD
:1005F000D3630000E46300001F030000C368F0B58C
:100600009D00836887B05D19030018330393036965
:1006100002909C00039B1F1943699E000093039B5B
:100620009E19D64B1B78002B0FD17F222B68D44903
:100630001C1213409B005B5800960435019235E074
:10064000CE4B1B78002B29D0009E029BCB4C9B6885
:1006500021780093EA1A029B92109B7812021A43A7
:10066000029B587802F0F6F90023029A2370137067
:1006700000960497029B039A9B68ED1A0193029BD4
:10068000AD10DD60049B9F1A029BBF101F61009B91
:100690009B1A029A9B10536101F077FB2B68019A19
:1006A0001C121340B64A9B009B5804359F46029B80
:1006B000587802F0C7F90023029A1370D9E7039B18
:1006C0003A1DD11AAD4B8B2903DD1A22009E1A70F8
:1006D000BBE71B783C60002B02D0009E1700B4E7FC
:1006E0002B6801991C120B40A5499B005B58170011
:1006F0000435DBE7039B3A1DD11AA04B8B2903DDA0
:100700001A22009E1A70A0E728681B78291D3860FD
:10071000002B03D0009E17000D0096E76B6801992F
:100720001C120B4096499B005B5817000835BDE72B
:10073000039B3A1DD11A914B8B2903DD1A22009E8F
:100740001A7082E7A4001B782C193C60002B02D0A1
:10075000009E170079E72B6801991C120B4088490D
:100760009B005B5817000435A0E7039B3A1DD11A84
:10077000824B8B2903DD1A22009E1A7065E781489F
:10078000A40021581B783960002B02D0009E17006E
:100790005BE72B6801991C120B4079499B005B5861
:1007A0001700043582E73A1F764B1168A400E15028
:1007B000724B1B78002B02D0009E170045E72B6878
:1007C00001991C120B406E499B005B5817000435C1
:1007D0006CE76C4BA600F058FFF766FE043F040080
:1007E0003868FFF761FE24180120664B640004435B
:1007F000F450624B1B78002B01D0009E25E72B683C
:10080000019A1C1213405E4A9B009B5804354DE729
:10081000039B3A1DD11A594B8B2903DD1A22009EE6
:100820001A7012E70098039C0121A04202D901002E
:100830000C3909681B783960002B02D0009E170024
:1008400003E72B6801991C120B404D499B005B5834
:10085000170004352AE7039B3A1DD11A474B8B2911
:1008600003DD1A22009E1A70EFE600990398814278
:100870000AD90B000C3B1B6843495B106418E41A4F
:10088000009BA400E35802E01821197000233B608C
:100890003A4B1B78002B02D0009E1700D5E62B6840
:1008A00001991C120B4036499B005B581700043518
:1008B000FCE6009B039A93420CD90C3B1968324B1F
:1008C0003A1FE3184910591A1068009B8900C85054
:1008D000170002E01822294B1A70284B1B78002BB6
:1008E00001D0009EB1E62B68019A1C121340244AE5
:1008F0009B009B580435D9E6009B039A934220D96C
:10090000009E214B0C3EE31804933368049A5B105D
:10091000D31A009A9B009858FFF7C6FD3C1F05901C
:100920002068FFF7C1FD3168049B4910591A059BE7
:1009300089001F1801207F00009B0743CF5027002C
:1009400002E018220D4B1A700C4B1B78002B01D0C3
:10095000009E7AE62B68019A1C121340084A9B00FD
:100960009B580435A2E6039B3A1DD11A034B8B29F1
:100970000CDD1A22009E1A7067E6C046F0000020C7
:10098000C8610000081A0020FDFFFF3F0099A40085
:1009900061581B783960002B02D0009E170054E686
:1009A0002B6801991C120B40CD499B005B58170026
:1009B00004357BE63A1F009B1168A400E150C94B47
:1009C0001B78002B02D0009E17003EE62B68019991
:1009D0001C120B40C2499B005B581700043565E6AA
:1009E000009BA4001C192368043F38685E10FFF7C1
:1009F0005BFD36180120BB4B76001B780643266052
:100A0000002B01D0009E20E62B68019A1C12134097
:100A1000B34A9B009B58043548E6039BA4003F1B48
:100A2000B04CBB420DD82378002B01D0009E0CE6C1
:100A30002B68019A1C121340A94A9B009B5804354D
:100A400034E6A94801F012FA2378002B01D0009E69
:100A5000FBE52B68019A1C121340A14A9B009B588E
:100A6000043523E6A300ED18002C00DA01E69D4BC7
:100A70001B78002B01D0009EE7E52B68019A1C1221
:100A80001340974A9B009B5804350FE63B1F049385
:100A90001B680593042B04D1A300ED18002C00DA89
:100AA000E8E5904B1B78002B02D0009E049FCCE51C
:100AB0002B68019A1C121340894A9B009B58049F83
:100AC0000435F3E53B1F04931B680593002B04D109
:100AD000A300ED18002C00DACCE5824B1B78002B2C
:100AE00002D0009E049FB0E52B68019A1C121340AF
:100AF0007B4A9B009B58049F0435D7E53A1F136837
:100B00005B10013B002B07DD01215B00A4000B43C0
:100B100004972D191360ADE5724B17001B78002B5D
:100B200001D0009E91E52B68019A1C1213406C4A7B
:100B30009B009B580435B9E53A00039B0C32D31A4D
:100B40008B2B04DD1A22674B009E1A707DE5FF2374
:100B500061005B000B4001210B433B60029B03984B
:100B60009B6824120493ED1A029BAD109B782D0212
:100B70001D43009B8D401B1A9B108B400B43BB6099
:100B8000029B0D437D609C70E4B2584BE4000299D7
:100B9000E35816008B6053490978002903D00833C5
:100BA0001D00170051E51D0001999B680C351C12B2
:100BB0000B404B499B005B580092170076E53B1FAA
:100BC0001E68039A009B93422AD104970A20F307D8
:100BD00016D4B3070DD1042E0BD90F23326813405E
:100BE000042B06D1300001F0CBF904F083FC063071
:100BF00006E00720042E03D0002E01D080208000C4
:100C0000643001F057FD002801D1043D32E5029B1C
:100C10003100587801F030FF0023029A137029E563
:100C2000009B009A0C3B1B6802995B109B005B4287
:100C30001C00D3180C3B1E601300083B1B68083CCB
:100C400017195A108A70D2B22849D2005B00555841
:100C50009B0A029A9B009560ED18009B043B1E685E
:100C6000039B7610B6009E191E4B1B78002B00D0FC
:100C7000EBE42B68019A1C121340194A9B009B5805
:100C80000096043512E53B1F1868FFF70DFCA40021
:100C900006003F1B1E2818DC02F068FC083E3618D0
:100CA00002F064FC124B801B9842F9D80D4B1B7864
:100CB000002B01D0009EC8E42B68019A1C1213403F
:100CC000074A9B009B580435F0E40123029A1370F5
:100CD00002F04CFC029B113886195E60C9E4C046E4
:100CE000C8610000F0000020F8630000101200202E
:100CF0009F8601003B1F1868FFF7D6FBA4003B1B33
:100D00000493BE4B061E9E4209DC0123029A137017
:100D100002F02CFCFA239B005E43113E04E0022308
:100D2000029A137002F02CFC029B36185E60A1E45C
:100D3000A300FF1A002320001A003900FFF7ECFB84
:100D4000AF4EB04C3168200001F04EFE31682000FB
:100D500001F099FEAC4B1B78002B01D0009E74E48F
:100D60002B68019A1C121340A84A9B009B5804351B
:100D70009CE4A54BA4001B783F1B002B01D0009ED8
:100D800063E42B68019A1C121340A04A9B009B58F5
:100D900004358BE401F0D4FC00F0F7FF3B1F18682A
:100DA000002823D1083B1868C30701D5401016E07E
:100DB00083070FD104280DD90F2302681340062B97
:100DC00002D1FFF77FFB0AE0052B03D1FFF77AFB87
:100DD000800004E019228C4B009E1A7035E43A0022
:100DE00001214300083A0B43136001E04010013831
:100DF000002832DD012243001343391F0B603B0002
:100E0000083B1B681341181A3B000C3B1B6813423C
:100E100003D08018A400904015E0990717D1042B47
:100E200015D90F211E683140062906D101308000F6
:100E3000C358009AA400A35010E0052907D1181840
:100E40000079A4004000009B1043E05006E0192206
:100E50006D4B009E1A70FFF7F8FB04356A4B1B7848
:100E6000002B02D0009EFFF7F0FB2B68019A1C12AA
:100E70001340664A9B009B58043517E4A300039A6D
:100E8000FB189B1A8B2B01DC002205E01A225E4B1B
:100E9000009E1A70FFF7D9FB631E002C03DD3A6039
:100EA0001C000437F8E7584B1B78002B02D0009E3B
:100EB000FFF7CBFB2B68019A1C121340534A9B008F
:100EC0009B580435FFF7F2FB3B00083B1868FFF71F
:100ED000EBFA3B1F04901868FFF7E6FA049AA600A5
:100EE000BC1B0023824200DA04332360464BBC1B48
:100EF0001B78271D002B02D0009EFFF7A6FB2B6856
:100F0000019A1C121340414A9B009B580435FFF77D
:100F1000CDFBA300FE1A04933B00083B1868FFF7C3
:100F2000C3FA3B1F04001868FFF7BEFAE20FC317AD
:100F3000A04253419B003360049BFC1A324B271D97
:100F40001B78002B02D0009EFFF77FFB2B68019AD5
:100F50001C1213402D4A9B009B580435FFF7A6FB3B
:100F60003B00083B18683B1F1968A300884202D168
:100F7000FB1A042222E004281ED90122104201D0CB
:100F8000114219D10326304215D10F2302681A40AD
:100F9000042A10D131420ED104290CD90A68134019
:100FA000042B08D1FFF79AFA431E9841A600BE1BF6
:100FB0008000306003E0A3000022FB1A1A60124B8D
:100FC000A4001B783C1B271D002B02D0009EFFF7BE
:100FD0003CFB2B68019A1C1213400C4A9B009B5847
:100FE0000435FFF763FB3B00083B18683B1F19689B
:100FF000A30088420CD1FB1A00222DE0E703000079
:10100000F8000020FC000020F0000020C861000073
:1010100004281FD90122104201D011421AD10326FF
:10102000304216D10F2302681A40042A11D13142EE
:101030000FD104290DD90A681340042B09D1FFF7F9
:101040004DFA030058425841A600BE1B8000306094
:1010500003E0A3000422FB1A1A60EA4BA4001B78E9
:101060003C1B271D002B02D0009EFFF7EEFA2B68D9
:10107000019A1C121340E44A9B009B580435FFF769
:1010800015FBA300FE1A04933B00083B1868FFF70A
:101090000BFA3B1F04001868FFF706FAE217C30FAC
:1010A000844253419B003360049BFC1AD54B271D9F
:1010B0001B78002B02D0009EFFF7C7FA2B68019A1D
:1010C0001C121340D04A9B009B580435FFF7EEFAE0
:1010D0003B00083B1868FFF7E7F93B1F04901868CE
:1010E000FFF7E2F9049AA600BC1B0023824200DD50
:1010F00004332360C34BBC1B1B78271D002B02D07D
:10110000009EFFF7A2FA2B68019A1C121340BE4AF8
:101110009B009B580435FFF7C9FA3B1F1B68B94A6F
:10112000A400042B02D13B1B002103E0002B03D1C0
:1011300004213B1B196001E00C23137013783C1B46
:10114000271D002B02D0009EFFF77FFA2B68019A23
:101150001C121340AC4A9B009B580435FFF7A6FABB
:10116000A300FC1A04933B00083B1868FFF79CF9A6
:101170003B1F06001868FFF797F936180120049BFB
:10118000760006432660FC1A9E4B271D1B78002B19
:1011900002D0009EFFF759FA2B68019A1C121340E7
:1011A000994A9B009B580435FFF780FAA300FE1A6A
:1011B00004933B00083B1868FFF776F93B1F0400D7
:1011C0001868FFF771F9241A0120049B6400044396
:1011D0003460FC1A8B4B271D1B78002B02D0009E1D
:1011E000FFF733FA2B68019A1C121340864A9B00C2
:1011F0009B580435FFF75AFAA300FC1A04933B00EE
:10120000083B1868FFF750F93B1F06001868FFF706
:101210004BF946430120049B760006432660FC1AE6
:10122000784B271D1B78002B02D0009EFFF70DFA8C
:101230002B68019A1C121340734A9B009B5804357B
:10124000FFF734FA3B00083B1868FFF72DF93B1F06
:1012500004901868FFF728F90100049803F086FB52
:10126000012340001843674BA4001B783E1B3060ED
:10127000371D002B02D0009EFFF7E7F92B68019A7B
:101280001C121340604A9B009B580435FFF70EFA6E
:101290003B00083B1868FFF707F93B1F04901868EC
:1012A000FFF702F90100049803F046FC012349000E
:1012B0001943544BA4001B783E1B3160371D002B93
:1012C00002D0009EFFF7C1F92B68019A1C1213404F
:1012D0004D4A9B009B580435FFF7E8F93B1F1868FF
:1012E000FFF7E2F8C317C018584001234000184325
:1012F000444BA4001B783E1B3060371D002B02D0EE
:10130000009EFFF7A2F92B68019A1C1213403E4A77
:101310009B009B580435FFF7C9F9A300FE1A0593FB
:101320003068012C03D1FFF7BFF8049008E0FFF705
:10133000BBF804007068FFF7B7F80130031B049393
:10134000049B002B01DC0123049304F029F8049989
:1013500003F0F2FB0C190121059B64000C4334607F
:10136000FC1A284B271D1B78002B02D0009EFFF78C
:101370006CF92B68019A1C121340234A9B009B585E
:101380000435FFF793F9A4003E1B3000FFF734F853
:101390001C4B30601B78371D002B02D0009EFFF7DE
:1013A00054F92B68019A1C121340174A9B009B5852
:1013B0000435FFF77BF9A300FE1A04933B00083BBA
:1013C0001868FFF771F83B1F04001868FFF76CF806
:1013D00004400120049B640004433460FC1A094B60
:1013E000271D1B78002B02D0009EFFF72EF92B68DB
:1013F000019A1C121340044A9B009B580435FFF7C6
:1014000055F9C046F0000020C8610000A300FC1A96
:1014100004933B00083B1868FFF746F83B1F0600A3
:101420001868FFF741F806430120049B7600064345
:101430002660FC1ADE4B271D1B78002B02D0009E75
:10144000FFF703F92B68019A1C121340D94A9B003D
:101450009B580435FFF72AF9A300FC1A04933B00BC
:10146000083B1868FFF720F83B1F06001868FFF7D5
:101470001BF846400120049B760006432660FC1AB8
:10148000CB4B271D1B78002B02D0009EFFF7DDF809
:101490002B68019A1C121340C64A9B009B580435C6
:1014A000FFF704F93B1F1868FEF7FEFFC043012356
:1014B00040001843BE4BA4001B783E1B3060371D14
:1014C000002B02D0009EFFF7C0F82B68019A1C1277
:1014D0001340B84A9B009B580435FFF7E7F8A30078
:1014E000FE1A04933B00083B1868FEF7DDFF3B1F24
:1014F00004001868FEF7D8FF8440012364001C43F1
:10150000049B3460FC1AAA4B271D1B78002B02D0C9
:10151000009EFFF79AF82B68019A1C121340A54A07
:101520009B009B580435FFF7C1F8A300FE1A0493F3
:101530003B00083B1868FEF7B7FF3B1F0400186824
:10154000FEF7B2FF0441012364001C43049B346096
:10155000FC1A974B271D1B78002B02D0009EFFF72B
:1015600074F82B68019A1C121340924A9B009B58F6
:101570000435FFF79BF8A4003E1B3000FEF757FE32
:101580008B4B30601B78371D002B02D0009EFFF77D
:101590005CF82B68019A1C121340864A9B009B58EA
:1015A0000435FFF783F8A4003E1B3000FEF74FFE22
:1015B0007F4B30601B78371D002B02D0009EFFF759
:1015C00044F82B68019A1C1213407A4A9B009B58DE
:1015D0000435FFF76BF8A4003F1B3800FEF749FE07
:1015E000734B1B78002B02D0009EFFF72EF82B6860
:1015F000019A1C1213406F4A9B009B580435FFF759
:1016000055F8A4003E1B3000FEF765FE684B3060C5
:101610001B78371D002B02D0009EFFF716F82B68B1
:10162000019A1C121340634A9B009B580435FFF734
:101630003DF8A4003F1B3800FEF784FE5C4B1B788E
:10164000002B02D0009EFFF700F82B68019A1C12B5
:101650001340584A9B009B580435FFF727F8A40015
:101660003E1B3000FEF7A8FE514B30601B78371D43
:10167000002B02D0009EFEF7E8FF2B68019A1C1297
:1016800013404C4A9B009B580435FFF70FF8039A10
:101690003B1D0493464C9B1A8B2B04DD1A23009EA2
:1016A0002370FEF7D2FF01F06BFF012340001843C7
:1016B00023783860002B03D0009E049FFEF7C5FFFF
:1016C0002B68019A1C1213403A4A9B009B58049FB6
:1016D0000435FEF7EBFF039A3B1D0493344C9B1A31
:1016E0008B2B04DD1A23009E2370FEF7AEFF01F062
:1016F0003DFF314B400018400123184323783860E8
:10170000002B03D0009E049FFEF79FFF2B68019AD9
:101710001C121340274A9B009B58049F0435FEF778
:10172000C5FFA4003E1B3000FEF78AFE204B306050
:101730001B78371D002B02D0009EFEF786FF2B681A
:10174000019A1C1213401B4A9B009B580435FEF75C
:10175000ADFFA4003F1B3800FEF78AFE144B1B7838
:10176000002B02D0009EFEF770FF2B68019A1C121E
:101770001340104A9B009B580435FEF797FFA300C7
:10178000FB1A0493012320001A000499FEF7C4FEFB
:101790000A4C2068643000F08DFF002800D1AFE2D1
:1017A000029B21685A78064801F07BF91EE0C0468A
:1017B000F0000020C8610000FEFFFF7FF80000205D
:1017C000FC000020A300FB1A049320000123002248
:1017D0000499FEF7A1FEE34C2068643000F06AFF34
:1017E000002800D18CE2E04801F07EF80223029A42
:1017F000137001F0C5FE236805331818029B58606A
:10180000FEF738FFA4003E1B300001F0D9FED74B95
:1018100030601B78371D002B02D0009EFEF715FFAD
:101820002B68019A1C121340D14A9B009B58043527
:10183000FEF73CFFA4003E1B300001F0C3FECB4B83
:1018400030601B78371D002B02D0009EFEF7FDFE96
:101850002B68019A1C121340C54A9B009B58043503
:10186000FEF724FFA4003E1B300001F0ADFEBF4B8D
:1018700030601B78371D002B02D0009EFEF7E5FE7E
:101880002B68019A1C121340B94A9B009B580435DF
:10189000FEF70CFFA4003F1B380001F0B3FEB34B72
:1018A0001B78002B02D0009EFEF7CFFE2B68019A1A
:1018B0001C121340AE4A9B009B580435FEF7F6FEFF
:1018C000A4003E1B300001F0BFFEA84B30601B7827
:1018D000371D002B02D0009EFEF7B7FE2B68019A41
:1018E0001C121340A24A9B009B580435FEF7DEFEF3
:1018F000A4003F1B380001F0D9FE9C4B1B78002B45
:1019000002D0009EFEF7A1FE2B68019A1C12134024
:10191000974A9B009B580435FEF7C8FE0121200022
:1019200001F0ACFE914B1B78002B02D0009EFEF71D
:101930008CFE2B68019A1C1213408D4A9B009B5809
:101940000435FEF7B3FE0021200001F097FE874B1F
:101950001B78002B02D0009EFEF777FE2B68019AC1
:101960001C121340824A9B009B580435FEF79EFED2
:10197000A4003E1B300001F0CDFE7C4B30601B7894
:10198000371D002B02D0009EFEF75FFE2B68019AE8
:101990001C121340764A9B009B580435FEF786FEC6
:1019A000A4003E1B300001F0C9FE704B30601B7874
:1019B000371D002B02D0009EFEF747FE2B68019AD0
:1019C0001C1213406A4A9B009B580435FEF76EFEBA
:1019D000A4003F1B380001F075FE644B1B78002B00
:1019E00002D0009EFEF731FE2B68019A1C121340B4
:1019F0005F4A9B009B580435FEF758FEA4003F1B2E
:101A0000380001F047FF594B1B78002B02D0009E95
:101A1000FEF71BFE2B68019A1C121340544A9B00D0
:101A20009B580435FEF742FEA4003E1B300001F037
:101A300071FF4E4B30601B78371D002B02D0009E8B
:101A4000FEF703FE2B68019A1C121340484A9B00C4
:101A50009B580435FEF72AFEA4003F1B380001F016
:101A6000DBFE424B1B78002B02D0009EFEF7EDFD03
:101A70002B68019A1C1213403D4A9B009B58043569
:101A8000FEF714FEA4003E1B300001F0DBFE374BD6
:101A900030601B78371D002B02D0009EFEF7D5FD6D
:101AA0002B68019A1C121340314A9B009B58043545
:101AB000FEF7FCFDA4003F1B380001F0BFFB2B4BE1
:101AC0001B78002B02D0009EFEF7BFFD2B68019A09
:101AD0001C121340264A9B009B580435FEF7E6FD76
:101AE000A4003F1B380001F0B5FB204B1B78002BF6
:101AF00002D0009EFEF7A9FD2B68019A1C1213402C
:101B00001B4A9B009B580435FEF7D0FDA4003F1BE9
:101B1000380001F0ABFB154B1B78002B02D0009E68
:101B2000FEF793FD2B68019A1C121340104A9B008C
:101B30009B580435FEF7BAFDA4003F1B380001F0A6
:101B4000B1FB0A4B1B78002B02D0009EFEF77DFDF7
:101B50002B68019A1C121340054A9B009B580435C0
:101B6000FEF7A4FDF8000020FC000020F00000209B
:101B7000C8610000A4003E1B300001F069FF844BE7
:101B800030601B78371D002B02D0009EFEF75DFDF4
:101B90002B68019A1C1213407E4A9B009B58043507
:101BA000FEF784FDA4003E1B300001F059FF784B86
:101BB00030601B78371D002B02D0009EFEF745FDDC
:101BC0002B68019A1C121340724A9B009B580435E3
:101BD000FEF76CFDA4003E1B300001F049FF6C4B8A
:101BE00030601B78371D002B02D0009EFEF72DFDC4
:101BF0002B68019A1C121340664A9B009B580435BF
:101C0000FEF754FDA4003E1B300001F029FE604B9E
:101C100030601B78371D002B02D0009EFEF715FDAB
:101C20002B68019A1C1213405A4A9B009B5804359A
:101C3000FEF73CFDA4003F1B380001F04FFB544B66
:101C40001B78002B02D0009EFEF7FFFC2B68019A48
:101C50001C1213404F4A9B009B580435FEF726FD8B
:101C6000A300FF1A3900200001F01AFC484B1B7832
:101C7000002B02D0009EFEF7E8FC2B68019A1C1294
:101C80001340444A9B009B580435FEF70FFDA40007
:101C90003E1B300001F0D0FB3D4B30601B78371D00
:101CA000002B02D0009EFEF7D0FC2B68019A1C127C
:101CB0001340384A9B009B580435FEF7F7FCA300FD
:101CC000FF1A3900200001F07DFB314B1B78002BFF
:101CD00002D0009EFEF7B9FC2B68019A1C1213403B
:101CE0002C4A9B009B580435FEF7E0FCA4003B1BEC
:101CF0001800049301F066FD01F069FD002802D18F
:101D0000043DFEF7B6FC224B1B78002B03D0009E4F
:101D1000049FFEF79AFC2B68019A1C1213401D4A7F
:101D20009B009B58049F0435FEF7C0FCA4003E1B9B
:101D3000300001F04EFD164B30601B78371D002B34
:101D400002D0009EFEF781FC2B68019A1C12134002
:101D5000104A9B009B580435FEF7A8FCA300FF1A0D
:101D60003900200001F03BFD094B1B78002B02D00D
:101D7000009EFEF76AFC2B68019A1C121340054A6C
:101D80009B009B580435FEF791FC07B0F0BDC046A0
:101D9000F0000020C8610000014B1870002070475F
:101DA000F0000020F0B50023A02787B05A1E04924F
:101DB000002B05DC01F0F6F800F098FE19230493DF
:101DC000002503950295254B19688D4201DB049B84
:101DD000ECE7234B1A680132914200DC00221A60C2
:101DE0001B68204E01937B439A199B5D059234003A
:101DF000032B01D110002CE0002B2DD0012B0CD196
:101E0000029B002B02D101F0B1FB0290019A0299D2
:101E10007A43A4186368CB1A0FE0022B12D1039BFC
:101E2000002B02D101F0ACFB0390019A03997A4395
:101E3000A4186368CB1A9B029B0A0B498B4201D8FA
:101E40000323B354019B074A7B439B5C032B03D1C1
:101E50000598FEF7D3FBBAE70135B4E7F40000209C
:101E600000000020D00B00209F86010000B59BB031
:101E70000200054901A803F013FB01A800F034FD9E
:101E800000F034FEFCE7C0460864000037B5174D8B
:101E900004002868002801D002F0F6FEA40020000B
:101EA00002F0E8FE2860002801D1114809E001ABEA
:101EB000984208D20F4B02196B440193934202D20D
:101EC0000D48FFF7D3FF042802D808302860083CEB
:101ED0002B680A4A1C191360094B01211C6000235E
:101EE000084AD1500433642BFBD137BD24040020B1
:101EF000196400001CFCFFFF496400001C04002062
:101F000020040020081A002070B50D4D0D4E2B68DE
:101F10004C1CA40036681C19B44203D90A20FFF7F0
:101F20003BFF0BE02C601D00AC4201D904C5FBE770
:101F30000F220901104008431860180070BDC04608
:101F40001C040020200400200322CB1C70B50C00D0
:101F5000D9171140C9180500891000220420FFF785
:101F6000D3FF0023A34204DAE95CC21811710133E4
:101F7000F8E7E1430023C917214041180B7170BDF8
:101F800010B5830706D1042804D90F2304C81340D1
:101F9000042B03D00E20FFF7FFFE014810BDC04602
:101FA0005065000030B502248025094B094AED0038
:101FB0009C505C59002CFCD0A124E400884204D23F
:101FC0008025ED0018514019F8E70021995030BDE7
:101FD00000E001400405000010B5002804D1902065
:101FE00092210002890203E0922080218002C9022E
:101FF000FFF7D8FF10BD002802D092239B0201E01A
:1020000090231B021B6800201A0E532A01D11B02C9
:10201000180A704730B501248025064A064BED00AA
:10202000D4505459002CFCD001600021014AD150F9
:1020300030BDC04600E001400405000010B5002896
:1020400002D09220800201E090200002A623090223
:10205000DB05090A1943FFF7DDFF10BDF0B50124C8
:10206000802503000F4F08000F49ED007C507C597C
:10207000002CFCD09C46002810DD5478167893780C
:10208000240234431B0423431C00D37801381B066D
:102090002343644608C40432A446ECE700237B5083
:1020A000F0BDC04600E001400405000070B5050029
:1020B0004B680A009C1C2100FFF7D0FFA0002818E5
:1020C00070BD0000154B1B68002B04D080219223AB
:1020D000C9029B0203E09221902389021B0200287F
:1020E00007D1191D5B6802001B0E522B14D10A0088
:1020F00012E0002281420FD903681B0E522B0BD134
:10210000436802339B00C318994205D91A68110E1F
:102110000022522900D11A00100070472806002022
:102120008022F0B5520085B00021624802F0BFFD68
:10213000802200215200604802F0B9FD5F4B1B680D
:102140001A00029353425A4110000392FFF744FFD2
:10215000029B002B01D15A4C00E05A4C0020FFF7A3
:10216000B1FFFF270500002D00D194E02B681A1263
:102170001B143A403B4001921A000A3A092A43D8FC
:102180004C4B019A995C002900D07FE010224E4808
:1021900002F08DFD2E00336801991A123A409142E7
:1021A00017D11A143A400B2A06D0132A0CD00A2A47
:1021B0000FD1454B1E600CE03B40022B09DC424A2C
:1021C0009B00D3185E6004E0102200213E4802F01C
:1021D0006EFD3000FFF776FF061EDCD13A4B196822
:1021E00000290FD02000FFF761FF0400374E31684F
:1021F000002903D02000FFF759FF0400344B0436B8
:10220000B342F4D12B4B3EE0143B092B3ED82A4B72
:10221000019A995C002939D108222E4802F047FD25
:102220002E0033681A143A40152A0BD01D2A11D0FB
:10223000142A14D1019A1B123B409A420FD1254B0C
:102240001E600CE0019A1B123B409A4207D1214BC1
:102250005E6004E0082200211E4802F028FD3000E4
:10226000FFF730FF061EDCD11A4E3168002909D075
:102270002000FFF71BFF71680400002902D0FFF760
:1022800015FF04000C4B0121019A99542800FFF717
:1022900019FF050067E70298FFF7ADFE411C0398A0
:1022A000FFF7CCFE054B039A1A600B4B1C6005B080
:1022B000F0BDC04628050020280400202806002084
:1022C00004480200049000006C1A0020701A0020DC
:1022D0007C1A00207C1A00202C06002070B50020FB
:1022E000FFF789FE04000120FFF785FE844200DA33
:1022F00004000A4B1E687542754128001D60FFF7F7
:102300006BFE002E01D0064B00E0064B064A28006B
:10231000611C1360FFF792FE70BDC04628060020C6
:1023200004900000044802002C060020F8B50020AC
:10233000FFF761FE07000120FFF75DFE3E00224D22
:102340000643224C0CD180219020C9020002FFF7E5
:1023500029FE01213000FFF771FE2E601C4B2FE09B
:10236000874208DD002392212B60194B89022360EC
:102370002368002011E0012380212B60154BC90246
:102380002360F5E71A68551C18D0120E522A07D19F
:1023900001205A68023292009B188B42F2D311E05E
:1023A000002800D023600C4C0C49200003F09AF860
:1023B000200001F0EBF8FFF791FF04E0002802D0C5
:1023C000236000E02160F8BD280600202C060020D4
:1023D0000490000004480200841E0020C164000034
:1023E000F0B585B0039203220333DC171440294E65
:1023F000E3189C10336801900291002B02D08022D8
:10240000D20201E092229202234FA51C3B68AD004C
:102410005B199A4217D2FFF783FE3368002B02D074
:102420008022D20201E0922292023B685B199A421A
:1024300009D21A4C1A49200003F054F8200001F088
:10244000A5F8002023E0029B3E681B06190C6B4692
:102450001A7BA423DB051343019A0B431104FF22CB
:102460001204114019433000FFF7D4FD3300301D32
:10247000083321000193FFF7CDFD01980A9A21004E
:10248000FFF7ECFD3000019B083D5D193D6005B094
:10249000F0BDC046280600202C060020841E002027
:1024A000EA64000070B59AB0FFF740FFFF221F4CAE
:1024B000D2000021200002F0FAFB0020FFF702FE0C
:1024C000FF25002600281AD003681A142A400A2A79
:1024D00008D11A122A40FF2A0ED0D200A1180B717F
:1024E000A05009E0132A07D11B122B40FF2B03D069
:1024F000DB00E2181671E650FFF7E4FDE2E7FF218A
:102500000200C900235808305D1EAB41D218884232
:10251000F8D1074901A802F0C3FF01A800F0E4F9CF
:10252000044800F0E1F91AB070BDC0461012002056
:102530001165000029650000044A05491368C85464
:1025400001339B059B0D13607047C046300A002085
:1025500030060020114A70B51368114C984211DA08
:1025600006193178451CFA39012905D8AB4205DD39
:10257000717801391F2901D92800EFE70100251AD8
:10258000461C02D10023136006E0665C6E540131E4
:102590008B42FADC181A106070BDC046340A002065
:1025A000841A002010B500F0E1FF064B1A68904233
:1025B00001D200221A601B68C01A034B834280417B
:1025C000404210BD380A0020204E000010B5094AD4
:1025D000094C1268236893420AD0084AD05C01F083
:1025E000E9F8012804D1236801339B059B0D236082
:1025F00010BDC046300A00203C0A002030060020F2
:1026000010B50400064B074A1B6812689B1ADB438F
:102610009B059B0DA34202DAFFF7D8FFF2E710BD3E
:10262000300A00203C0A0020F7B506000191151E73
:102630002FD05768B800441C0630FFF7E1FFFB209D
:10264000FFF77AFF1C20FFF777FFF0B2FFF774FF68
:10265000E0B22412FFF770FFE0B2FFF76DFF6B46A8
:102660001879FFF769FF0026BE4212DAB300EB18B3
:102670009C680136E0B2FFF75FFF2012C0B2FFF79F
:102680005BFF2014C0B2FFF757FF200EFFF754FF87
:10269000EAE7F7BDC82210B5D2000021034802F0D6
:1026A00006FB0022024B1A6010BDC046D00B002072
:1026B000F4000020064B074A1B6812689B1ADB4394
:1026C0009B059B0D0122834200DC00221000704715
:1026D000300A00203C0A0020F8B505000C00160066
:1026E0001F1E0ED10320FFF7E5FF002827D0FA2098
:1026F000FFF722FFE8B2FFF71FFFE0B2FFF71CFF72
:102700001DE0501DFFF7D6FF002818D0FB20FFF773
:1027100013FFE8B2FFF710FFE0B2FFF70DFFF0B2D2
:10272000FFF70AFF3012C0B2FFF706FF3C00E31BC1
:102730009E4204DD2078FFF7FFFE0134F7E7F8BD85
:1027400070B50024A0250B4B1B689C420EDA2A00B2
:102750006243094BD3181A78002A05D05978002310
:1027600011201A00FFF7B8FF0134ECE7FFF792FFE2
:1027700070BDC046F4000020D00B00200123F3B54B
:102780000400FFB00D0010001A420DD002AA137011
:10279000431002A9537042121B0E40148A700B7131
:1027A000C8700B00052273E0032313401ED1042AD6
:1027B0001CD90F2201680A40042A17D1023302AA49
:1027C0001370FFF7DDFB060002F094FEF823FF33E1
:1027D000984200DD18000023834205DA01335A1EB7
:1027E000B25C02A9CA54F7E7421C50E0042801D0A9
:1027F000002809D1032302AA04381370434243413D
:1028000053701300022243E0002B45D1042843D922
:102810000F2102681140052912D1043302A90B705F
:10282000F8231209FF3392009A4200DD1A000023B8
:1028300093422BDA0133C118C97802AEF154F7E79D
:10284000062929D101390E00120956430196F826AE
:10285000019FFF36B7421FDC02AE31700136934252
:1028600013DA0127013399004158394201D0394127
:1028700000E00A49012737700F127170B7700F140A
:10288000090EF77031710536E9E7019A013202ABA2
:1028900029002000FFF720FF7FB0F3BD19FCFFFFE8
:1028A00070B5A023050000240D4A1800604380186D
:1028B0004178A94203D001340A2CF6D10FE0A022BE
:1028C000002102F0F4F9074A1368013BA34200D14A
:1028D0001460002329001A001120FFF7FDFE70BDCF
:1028E000D00B0020F400002010B5B2B002236A46DD
:1028F0000400137002F0FEFDC72800DDC72000238E
:10290000834205DA694601335A1EA25CCA54F7E7CE
:10291000421C6B46FF211420FFF7DEFE32B010BDD3
:10292000F7B5234B06001B68A02000930023214924
:10293000009A93420ADA02005A438A185478B44241
:1029400002D11278002A32D10133F1E70024A0230A
:102950001A00624301920199164A55182F78002FE8
:1029600006D001340A2CF3D11348FFF7BDFF1EE057
:10297000A0223900280002F09AF903230D4A019998
:102980006E7053540D4BF200D358AE70AB600223FF
:10299000EB60009B2F616F61A34202DC044B0134AA
:1029A0001C60002331001A001020FFF795FEF7BDD0
:1029B000F4000020D00B0020E4650000101200207D
:1029C00010B5FFF7BDFE0024064BE200D3181B79BB
:1029D000043B012B02D8E0B2FFF7A2FF0134FF2C29
:1029E000F2D110BD10120020F8B507000D00002430
:1029F000134BE200D3181A79062A1DD118687932D0
:102A0000C3681A40042A17D11B0A01339B000C30FB
:102A1000C018FFF7B5FA060002F06CFD0023A842CB
:102A20000AD19D4205DDF15CFA5C914204D101338B
:102A3000F7E7E0B2FFF774FF0134FF2CD8D1F8BDFF
:102A400010120020002310B501001A001120FFF71A
:102A500043FE10BD07B56B46197069465A701312D4
:102A60008B701314120ECB700A716B460100052295
:102A70001320FFF731FE07BD10B50A000100122038
:102A8000FFF77CFE10BD70B5050008000C00323069
:102A9000FFF7B6FD2B00220000211B20FFF71CFED4
:102AA00070BD10B50C000300110014202200FFF7C8
:102AB00013FE10BD70B506000020FFF703FB0024D5
:102AC000FF25002810D003681A142A40152A05D1C2
:102AD0001B122B40B34204D1040002E01D2A00D196
:102AE0000024FFF7EFFAECE7200070BDF0B5802777
:102AF0009DB0FFF76BFDBC4CBC4D2068FF00391A40
:102B0000401900F03DFE23680600C3182360002B27
:102B100000D1F7E1002E0DDD2068391A281800F0E9
:102B20002FFE236806001B18236000F01FFDB04B2A
:102B30001860EFE72B78FA2B00D027E12368022BEF
:102B400006DCFFF72FFD002800D1DBE10120D4E1F6
:102B50006878AC780238182800D915E101F072FEC7
:102B600019002A002E0032003500390014014400FB
:102B70006E007D0083009700E800FD001401140141
:102B8000140114011401140114011401140114019D
:102B90000E01FF2C00D1F7E02000FFF781FE00229C
:102BA0009449E3005A50CB181A7121000092130087
:102BB00013204FE02000FFF7B3FEE5E02000FFF711
:102BC0006FFEE1E0FFF7FCFEDEE0FFF7B9FD8A48AB
:102BD000D1E0182C00D9D7E0884BA200D2582100B0
:102BE0001520FFF7CBFDCFE000242000FFF762FFA8
:102BF000071E03D10134192CF7D1C5E0083002F0CB
:102C000079FC06000530FFF7FBFCFB20FFF794FC86
:102C10001D20FFF791FCE0B2FFF78EFCF0B2FFF74A
:102C20008BFC3012C0B2FFF787FC0025AE42E1DD1D
:102C30007B19187AFFF780FC0135F7E700230121A3
:102C40006E4AD1500433642BFBD100211D200B00B0
:102C50000A000091FFF7C4FB96E0002221000092D9
:102C600013002720F6E700F099FC03AC644A6421C6
:102C70000090644B200002F0E1FB0223200023704F
:102C800002F038FC23000200002116207AE0002424
:102C9000584AE300D558002D46D06B689E00701D41
:102CA000FFF7AEFC2B000025320008332100012085
:102CB000FFF712FD0020FFF705FA2E002F00002875
:102CC0001DD0FF2103681A120A40A24214D11A141F
:102CD0000A400B2A07D10B400DD0012B09D0022B43
:102CE00000D10DE108E0132A06D100252E002F00A7
:102CF00002E0060000E00700FFF7E4F9DFE7002E3E
:102D000004D0320001212000FFF78EFC002D04D0FA
:102D10002A0002212000FFF787FC002F04D03A0090
:102D200000212000FFF780FC0134FF2CB0D12BE004
:102D3000FFF706FD0025002429000094230022004F
:102D400013200135FFF74CFBFF2DF4D1FF222100AA
:102D5000D200284801F0ABFF16E0FFF7F1FC00209D
:102D600000F078FA00F01EF900F0FCFCE120C00051
:102D7000FFF78CF82448FFF7B7FD05E000231A2081
:102D80001A001900FFF7A8FC0320B6E0FB2B00D0C7
:102D9000DCE62268042A00DCD3E62E79E8781B4BB7
:102DA000360206439E4200DDD0E6331D9A4200DC27
:102DB000C7E6EB5CFE2B00D0C8E66878AC78731EE3
:102DC0001C2869D007D8082836D01B285FD00128D6
:102DD00000D091E01CE01E2800D17FE067D31F28BF
:102DE00000D181E088E0C046340A0020841A002027
:102DF000380A002010120020F9650000081A00208F
:102E0000106600000B66000017660000F603000065
:102E1000FF2C71D02000FFF743FD6D793A4AB31EB5
:102E2000009221002A000A20FFF7DAFA374BE4006B
:102E3000E0501C1925715FE0182C5DD868790228D4
:102E400013D003281BD0012856D1AF1D7A78AD7955
:102E5000BB7812022A431B0413431A00FB78A40018
:102E60001B0613435B0003430EE0002B44DDB11E41
:102E70002548FFF769F8264BA400E0503CE0AB7909
:102E8000A4005A1E93419B00214AA35034E019002C
:102E90002048FFF7A9FD2FE0FF2C2DD06A79022AE8
:102EA0002AD81949B31E00910B20210022E0632B80
:102EB00000DD6323002203A8934204DDA9184979A9
:102EC00081540132F7E7D9430022C917194041184C
:102ED0000A7001330090210015200BE00D4A2100FB
:102EE00000921E20002205E0042B05D1094A210092
:102EF00000920022FFF774FA701DFFF72BFB01E030
:102F00000500F9E61DB0F0BD8A1A0020101200205D
:102F1000081A0020891A0020F0B5EFF31081012370
:102F2000194083F31088134E134AB4461268013ACD
:102F30009340124A1468124A1568124A002B15D0A1
:102F4000166803420BD02660C046C046C046C04645
:102F5000C046C046C046C04616682E6004E06746BC
:102F60003E601668084F3E605B08E7E781F3108813
:102F7000F0BDC0460805005004000020480A0020AB
:102F8000500A0020400A00200C05005010B5012412
:102F9000044001D0441002E00D20FEF7FDFE2000A9
:102FA00010BD0000F0B5A14F85B03B68002B04D1E7
:102FB0009F4A1268002A00D136E19E4D2A68002AF5
:102FC0002AD19B4E3468002C0FD1002B0DD00C322F
:102FD000994901A801F062FE6B460433185D012196
:102FE000013400F0DFFA0C2CF6D13368002B11D03D
:102FF0003C68002C0ED101AD0C228F4928003460B2
:1030000001F04CFE285D0021013400F0CBFA0C2CBD
:10301000F8D109E13B68336000211A2001F002F980
:1030200000211B2001F0FEF800211C2001F0FAF81D
:103030002E68012E56D0022E00D19CE0002E00D02A
:10304000ECE0013631007A4C03202368994301F00B
:10305000E9F80420216801400B005942594101F070
:10306000E1F8102123680A200B405942594101F030
:10307000D9F88021236809010B40594259410620A3
:1030800001F0D0F88021236809020B4059425941D0
:10309000072001F0C7F88021236849020B405942FC
:1030A0005941092001F0BEF88021236889020B40B4
:1030B00059425941192001F0B5F880212368C9020D
:1030C0000B4059425941182001F0ACF88023216887
:1030D0001B030B4059425941172001F0A3F831005E
:1030E0001A2099E00221524C172023680B405942C4
:1030F000594101F097F80821236818200B405942E4
:10310000594101F08FF880212368C9000B405942D2
:103110005941042001F086F88021236849010B40C1
:10312000594259410A2001F07DF880212368C901E4
:103130000B4059425941032001F074F88021236863
:1031400089030B4059425941092001F06BF8802353
:1031500021681B040B4059425941192001F062F8C3
:103160003100062001F05EF83100072001F05AF826
:1031700031001B2050E020212D4C172023680B40EC
:103180005942594101F04EF84021236818200B4064
:103190005942594101F046F88021236819200B401B
:1031A0005942594101F03EF88021236849000B4003
:1031B00059425941092001F035F8802123688900DE
:1031C0000B4059425941072001F02CF88021236817
:1031D00089010B4059425941062001F023F8802112
:1031E000236849030B40594259410A2001F01AF85B
:1031F00080212368C9030B4059425941032001F043
:1032000011F8802321685B040B4059425941042086
:1032100001F008F801211C2001F004F82B680321BB
:10322000581C01F089FC296005B0F0BD4C0A002053
:10323000440A0020540A00202F660000006810B5E0
:10324000C30703D5FFF7A2FE014B186010BDC046AF
:103250004C0A002013B5002401A8019400F032FAB2
:10326000014B1C6013BDC0464C0A002070B5050020
:103270000068FFF78BFE04006868FFF787FE631E97
:10328000042B0CD80138042809D805225043043AED
:10329000C3189A40130002490A6813430B6070BDBB
:1032A0004C0A002070B505000068FFF76FFE0400AF
:1032B0006868FFF76BFE631E042B0CD801380428E6
:1032C00009D805225043043AC3189A401300024912
:1032D0000A689A430A6070BD4C0A0020F7B5304A6C
:1032E0001368002B0CD12F4B196801238B402E49FA
:1032F0000B602E4911602E4A2E4911602E4A136030
:1033000001260468344219D0FF2263101802120407
:103310001040FF22611212020A40DBB21043184330
:10332000264B1B68202B06D1B440254BA40EA400CD
:10333000E35800021843FFF7EFFD30E00325254076
:103340002DD1042C2BD90F2322681340062B26D114
:10335000FF27130901933F04019B9D421FDAAB0035
:10336000E3185A68324218D0531018023840FF212F
:1033700084460902501208406146DBB208431843F4
:103380000E4B1B68202B06D15200920E0C4B920064
:10339000D35800021843FFF7BFFD0135DCE7F7BD46
:1033A000480A0020106A0000400A0020080500506A
:1033B000500A00200C0500501805005004000020A1
:1033C0003C660000012310B50C68134A234003D06B
:1033D0006310012804DC07E001281ADD01235B42A9
:1033E00048682021042800D018211160202B00D922
:1033F00000230A4A9B009A5801239340084A09492E
:103400001360094A1160094A09491160094A1360A9
:1034100010BD18211160ECE704000020106A0000C4
:10342000400A002008050050480A0020500A0020E9
:103430000C050050180500500068F8B5C30702D508
:10344000FFF7A4FD0BE0830726D1042824D90F221F
:1034500003681A40042A1FD11B091DD000790300FC
:10346000203B5E2B18D80522002053430B4E9D189D
:10347000043AAB420CD0052110249F5D3C4200D0A1
:1034800080180139520064100029F7D10133F0E7A8
:1034900001234000184300E00120F8BD3C67000014
:1034A000F0B5040085B008680E00FFF76FFD0190CD
:1034B000022C07DD7068FFF769FD0400B068FFF7B4
:1034C00065FD01E001200400174B011D1A6805236A
:1034D000461E43430120002784460291211D053BDF
:1034E000039102998E4219D0611E039DA94212D008
:1034F000042E0DD804290BD8019D5F18054203D076
:103500006546BD402A4302E06546BD40AA43012707
:1035100040000131E9E701360533E2E7002F01D031
:10352000014B1A6005B0F0BD4C0A002010B50A200E
:1035300000F0FEFC0023FF21024A995401331D2BA9
:10354000FBD110BD580A002001220020054B06497E
:103550001A615850033004315850801808315850BF
:103560001A60704700800040040500000122034BF0
:103570001A64A822D20098587047C04600800040C4
:1035800010B5FFF7F3FF800A10BD000010B5010071
:10359000014800F001FF10BD5C0B0020004870479F
:1035A0001769000070B5054E0400335C0D008B42B6
:1035B00002D000F019FE355570BDC046580A0020F3
:1035C0000D2070473B207047036870B55B100120E9
:1035D000052B12D8094A9B009C58094D2B5D002BE6
:1035E00005D00021200000F0FFFD00232B55200016
:1035F00000F0A4FC01234000184370BD24690000C2
:10360000580A002070B5036845685C106D1004D43A
:103610000B4B9D4202DD1D0000E000251C2C0DD847
:10362000084E335D012B05D00121200000F0DCFDA8
:10363000012333552900200000F00EFD70BDC04667
:10364000FF030000580A002070B5046864101C2CA9
:103650000FD8094D2B5D002B05D00021200000F074
:10366000C3FD00232B55200000F0F2FD04230128A8
:1036700000D00023180070BD580A002070B5040067
:103680000D001C280ED8084E335C012B04D00121FC
:1036900000F0AAFD01233355290020004D1EA94149
:1036A00000F0C0FD70BDC046580A0020436810B548
:1036B000191F4A424A41006811004010FFF7DEFF1F
:1036C00010BD000070B5124C0500A37E012B05D083
:1036D00001211A2000F088FD0123A3762379012B14
:1036E00005D00121042000F07FFD0123237128680B
:1036F000042804D1002100F095FD012104E00121FE
:10370000042000F08FFD00211A2000F08BFD70BD19
:10371000580A002010B5084C6379002B05D0002111
:10372000052000F061FD00236371052000F090FD8D
:1037300043425841800010BD580A002010B5084C83
:10374000E37A002B05D000210B2000F04DFD002373
:10375000E3720B2000F07CFD43425841800010BD15
:10376000580A0020E12110B54902044800F05BFE30
:10377000FFF7EAFEFFF7DAFE10BDC0465C0B002043
:10378000F8B50B4E070030000D0000F08BFE041E54
:10379000AC4200DD2C003D00EB1B9C4205DD3000FF
:1037A00000F08AFE28700135F6E72000F8BDC0461B
:1037B0005C0B002010B50100014800F03BFE10BD7D
:1037C0005C0B002010B51B20FEF7E6FA10BD0420AC
:1037D000704710B51B20FEF7DFFA012010BD10B5B1
:1037E0001B20FEF7D9FA10BD10B501210D20FFF7FF
:1037F000D9FE01210E20FFF7D5FE00210F20FFF793
:10380000D1FE044C200000F09FF91021200000F0B0
:10381000B7F910BD8C0A002010B504680D20E3072D
:1038200003D56410FF2C03D91720FEF7B5FA06E084
:10383000FFF7DAFFE1B2024800F0C4F9002010BD42
:103840008C0A002010B5FFF7CFFF0021034800F0DD
:10385000B9F901234000184310BDC0468C0A00206E
:103860000122094B1A60094A1368002BFCD003227D
:10387000074B1B68D8171040C0180123801006386A
:10388000400018437047C04600C0004000C10040DF
:1038900008C50040F7B501260468344205D04268E7
:1038A000324202D08368334201D10D2005E052102C
:1038B00064100092802C03D91520FEF76DFA23E0E6
:1038C000009A1620FF2AF8D85B1001931720FF2BCF
:1038D000F3D80E4F0E4D3B68002B03D1280000F0AB
:1038E000F7F93E60E1B2280000F080FA6B4628004C
:1038F000197800F0AEF96B462800197900F0A9F9A3
:10390000280000F0DDFA0020FEBDC0467C0A002041
:10391000A00A0020F7B501260468344202D04168AD
:10392000314201D10D2005E04B1064100193802C31
:1039300003D91520FEF730FA2EE0019B1620FF2B4D
:10394000F8D8164F164D3B68002B03D1280000F025
:10395000BFF93E60E4B22100280000F047FA6B4650
:103960002800197900F075F90021280000F04AFAC2
:10397000002801D040420CE001222100280000F084
:1039800030FA280000F05BF90028FAD0280000F097
:103990005BF9012340001843FEBDC0467C0A0020AD
:1039A000A00A0020F8B5274B06001A681F00264C15
:1039B000002A19D1254D2B68002B04D1200000F0DE
:1039C00087F901232B601D21200000F00FFA2A2126
:1039D000200000F03EF90121200000F03AF920001B
:1039E00000F06EFA01233B601D21200000F0FEF97B
:1039F000F1B2200000F02DF90021200000F002FAC1
:103A00000300002083421BD101221D21200000F071
:103A1000E8F9200000F013F90028FAD0200000F0A7
:103A200013F97F2801DD0138FF3803007F3301DA05
:103A30007F20404264237F215843494200F096FF93
:103A4000F8BDC046780A0020A00A00207C0A0020A9
:103A500010B50120FFF7A6FF01234000184310BD59
:103A600010B50320FFF79EFF01234000184310BD4F
:103A700010B50520FFF796FF01234000184310BD45
:103A800010B5FFF76FFEE120C000FEF7FFF9044814
:103A9000FEF72AFFFEF706FDFEF792FF10BDC046B7
:103AA0001766000010B5FEF77DF910BD70B5002552
:103AB00004AC24780573A94205D10A4B0A4A232194
:103AC0000A4801F06BF801600949920052589B00C6
:103AD00002715B588371A3005B58856043710223B8
:103AE000C37170BD796900003C69000087690000FE
:103AF000106A0000037B002B04D1437383730361BE
:103B000001330373704700001FB50191A021002409
:103B10000068C900D2B24450012A07D0A24203D0A3
:103B2000032A05D1042202E0022200E00622134308
:103B3000034A8350034B019AC250012343501FBDD7
:103B4000540500002405000010B50400FFF7D2FF63
:103B5000A1222368A179D20099506179064A2000F8
:103B60009950217904329950044B19685A689B681E
:103B7000FFF7CAFF10BDC0460C050000800A0020F8
:103B80004BB2002B0CDB80233F290CD81F290CD80B
:103B90000F290CD807290CD803290CD81B060BE0D9
:103BA00080239B0408E0DB0406E01B0504E05B05C2
:103BB00002E09B0500E0DB050168014A8B5070477D
:103BC000240500000368074A99501A00FC32D168A6
:103BD0000029FCD0A321C90058580023C0B2D360EB
:103BE0007047C0461C05000007B58022074BD20570
:103BF0001A6000229A6002321A710F230C3200936D
:103C00000349023B0348FFF751FF07BD800A00202C
:103C1000003000408C0A0020F8B505000E001700A7
:103C20000024BC4208D02B68315D1B6828009847EF
:103C3000002801D00134F4E72000F8BD704710B52A
:103C40001C3000F0D5FB10BD10B51C3000F0C2FBDD
:103C500010BD70B5437E0D00002B05D0643004000C
:103C600000F0D5FB002801D0002004E0200029004E
:103C700000F0A1FB012070BD10B51C3000F0BEFBB0
:103C800010BD0000F7B50193FA23002504009B0046
:103C900083600D4B4560083303601C300F00160035
:103CA00000F07EFB2000643000F07AFB074AB6008B
:103CB000B35827616375019B20009B009B58657674
:103CC000A576A375FEBDC046F0690000106A00002D
:103CD0000123A022C375837D0C49C133FF33D20574
:103CE0009B009950437DC133FF339B009950CC21F9
:103CF0000369074A490499500521243A9950817D66
:103D000008329950417D034A995070470C060000D3
:103D1000240500000C050000F7B5050000200C008C
:103D2000019382425CD0161E402E00D940262F00FF
:103D30001C37380000F04AFBB1222B69D2008021E9
:103D40009C50012289005A50A97E002901D11A6293
:103D50001A600024731E2A69A34206D1019B002B1E
:103D600003D0802302219B00D15001231362130052
:103D7000FC33D968002902D1996A0029F9D0996ADF
:103D800000290AD1D960A323DB00D1583800C9B279
:103D9000013400F010FBA642DCD8019A2B69002AFE
:103DA00004D11A00FC32916A00290AD001210022B4
:103DB000AA7659611900FC3188680028FCD08A6015
:103DC00007E00121A976D961D16C0029FCD000213E
:103DD000D164FC339A6A002A01D000229A62E0B2D0
:103DE000FEBD10B50123FFF797FF10BD0300AC33F4
:103DF00010B504001970643000F0E8FA012363760E
:103E000010BD0000F8B500220D0001004276AC3173
:103E1000036904000878B121C90058508021890045
:103E20005A5001321A629A6026006436300000F05F
:103E3000DFFA00280ED03000276900F0CBFA1E4BC5
:103E4000F8502369FC331A6A002A0CD19A6A002AB6
:103E5000F9D008E02369002D0AD11A00FC32916ADA
:103E6000002905D10EE09A6A002AF3D11A62DBE735
:103E700001225A611A00FC3291680029FCD000210D
:103E8000916006E00121D961D16C0029FCD00021AC
:103E9000D1641A000020FC32916A81420BD007499C
:103EA00090625A5802305A50824204D0043A534227
:103EB00053410230C01AF8BD1C050000C4040000C4
:103EC00010B50121FFF79EFF10BD000010B51323B0
:103ED000142202490248FFF7D5FE10BD0040004001
:103EE000A00A002003210A4802680A430260094828
:103EF00002680A4302600849084A094B9B1A03DD1D
:103F0000043BC858D050FBDC00F0B4F9FCF732F9A0
:103F10002405004054050040A86C0000000000206B
:103F2000D4000020FEE7FEE7FEE7FEE7FEE7FEE73F
:103F3000014B18607047C04610000020F7B5002301
:103F4000202877D83C4B8000C258042A14D006D8C9
:103F5000022A0DD00ED80423012A14D069E0062AC3
:103F60000ED00BD31A2A0DD002231B2A0BD060E0EF
:103F7000082308E0102306E0202304E0402302E0A9
:103F8000802300E001232D4A1268082A04D9092A57
:103F900005D00A21022404E00821002401E01100D8
:103FA0000124A02501261C272548ED004651254D5A
:103FB000254E2D681B02AD003D400195234D2D6817
:103FC00000958559AC466746214D3D401D438551BE
:103FD0008359C0259C46009BAD021D40FF236746C8
:103FE0001B023B402B43019D1D43009B5F0160234F
:103FF0001F402B003B431C4301238451154C03609D
:1040000063680F48002BFBD00024124B01255C6035
:10401000A123DB00C3584560A025ED0044511BB22D
:10402000914207D002D98A1AD34003E0521A934032
:1040300000E000231800FEBD106A000014000020FC
:10404000007000400C000020040500000800002063
:10405000FF00FFFFFC700040F0B520286CD8374B04
:104060008000C258364B1E68002E2ED1C22435481F
:10407000A4000759344B03253B40C0273F023B4374
:1040800003518023893C9B00FF3C03512F4F036069
:104090002F4B803CD859FF3CA043D8510437D85906
:1040A000A8432043D8510837D8590C35A843083DB8
:1040B0002843D851A820C0001E508026C120760277
:1040C00080001E501C601E4B1C60002314262148DB
:1040D00034005C43255804006F1C0FD11420584352
:1040E0002250A0200325C132FF329200C005155096
:1040F000194A08001268082A03D10BE0AA4218D115
:10410000ECE7082A02D9083AD14002E00820821AD6
:104110009140080014225343E3189A680C49513225
:10412000FF32920058605050DA68C1239B00CA5099
:1041300002E00133032BCBD1F0BDC046106A000072
:10414000580B002000E100E0FF00FFFF0405000025
:104150000090004018000020100000201E4BF0B519
:10416000596C18001D4A002914D0A025A12600234F
:104170000124ED05F600D1584F1C06D0D7187F68F2
:10418000002F02D027008F40AF5114333C2BF2D1C7
:1041900000234364131DA0254032944600200124CF
:1041A0000F4EED05DA680F49920057180A49521868
:1041B000526C002A0CD01A1F1268511C05D01968C5
:1041C000FF2902D021009140A9513A00FC325064ED
:1041D00014339C45E6D1F0BDFC900040180000204F
:1041E0000C0500000090004000B5202816D80C4AAD
:1041F00083009B58032911D8A0220800C133FF3344
:10420000D2059B0000F014FB02080406002104E024
:104210000C2102E0042100E00321D15000BDC04682
:10422000106A000020280DD8074B8000C058A0223B
:104230000123D2058340002901D1044901E0A121D5
:10424000C90053507047C046106A00000C050000BA
:1042500003000020202B0AD8A222A021D200C905E9
:104260008858034A9B009B58D84001231840704748
:10427000106A00002D4B10B51A78012A19D12C4A6A
:104280001268120715D12B4AE0241168F0220800A9
:10429000104021420BD128490968114209D1274910
:1042A000274A11608021274A0902116001E0302865
:1042B000F1D01A78012A0DD11D490968090709D1E1
:1042C000F0201C4909680140402903D11A490968B6
:1042D000014223D01B68DBB2012B25D1144B1B6894
:1042E0001B0721D1134B1A68F0231A40A02A04D1CE
:1042F000114A12681A4203D016E0D02A14D1F7E707
:10430000114B1A68012A03D1C022104B1A600BE02E
:104310000F4A1A601A68012AFCD1F5E7C1218020F2
:10432000C900C0054250D5E710BDC046E00F00F0FF
:10433000E40F00F0E80F00F0EC0F00F0DFFF07C023
:1043400004050040186C004000EC064014EC0640E8
:1043500075930000F7B506000D000C008B18019353
:10436000019B671B9C4207D0336821781B68300093
:10437000984701340028F3D13800FEBD70B5050020
:104380000C00081E07D001F0B5F82B6802005B682E
:1043900021002800984770BD10B5FFF7EFFF10BD52
:1043A00010B540220021040000F081FC0023200011
:1043B0002364636410BD3F23026C10B5541C23407A
:1043C000446C9C4201D08154036410BD00230364FB
:1043D00043647047436C026C934206D03F21C25C39
:1043E00001330B404364100001E00120404270475C
:1043F000036C406C181A00D540307047436C026C57
:10440000934201D0C05C01E0012040427047036C40
:10441000406C5A1C3F231340181A42424241D0B20A
:1044200070470120704710B503681322DB69984775
:1044300010BD70470369054A9950FC331A6A002A77
:10444000FCD0002201201A627047C0461C05000003
:10445000030010B55C331A781F23134001221100AA
:1044600099400D4B0424D967C221036989005C502F
:104470005A60DA60A0220021D20099500122074937
:1044800052425A50064914305A500C395A50083189
:104490005A50FFF79BFF10BD04E100E00C0500003F
:1044A0001405000010B51430FFF7A2FF10BD10B5C1
:1044B0001430FFF7A3FF10BD10B51430FFF78AFFCB
:1044C00010BD0000030070B55E331C780269604BBC
:1044D000D45003005D331C785E4BD450030061332D
:1044E0001C785D4B012C0CD105005F352E78A22580
:1044F000ED005651050060352E78A125ED0056518E
:1045000000E00024D4509623DB00994238D996234A
:104510001B01994237D996235B01994236D99623DC
:104520009B01994234D9E1239B01994232D99623C8
:10453000DB01994231D9E123DB0199422FD996233E
:104540001B0299422DD9E1231B0299422BD99623B4
:104550005B02994229D9E1235B02994227D9E123E1
:104560009B02994225D93D4B994224D9E123DB0294
:10457000994223D9E1231B03994221D8384B21E0EA
:104580009E23DB021EE09D231B031BE0354B19E03D
:10459000354B17E0EC239B0314E0344B12E0344B13
:1045A00010E0344B0EE0344B0CE0344B0AE0344B5B
:1045B00008E0344B06E08023DB0403E0324B01E0EB
:1045C00080235B0531490024535004232439535080
:1045D0001100FC31CC600C62C121013489001460EF
:1045E0005C309460535003781F202200D9B20840F9
:1045F000824080342648FF345BB20251002B13DA2C
:104600000F230B40083B234C9B089B001B190324E2
:104610002140A140FC348C40DD69A543C0248C407E
:1046200021002943D96111E0194C9B089B001B19FB
:1046300003242140A140C025FC348C40AD005E59CC
:10464000A643C0248C40210031435951026070BD03
:104650000C050000140500006C05000090D003005C
:1046600000D0BE0E00B013000050270000A04E0086
:1046700000F0750000509D0000F0EB0000903A0142
:1046800000E0D70100B0AF0300705F072405000011
:1046900000E100E000ED00E0F7B5009308AB1B7807
:1046A00000250193FA2304009B0083600E4B4560B4
:1046B0000833036014300F001600FFF771FE23006B
:1046C0005C3327611E70009B084A9B0099582300A9
:1046D0005D331970019B20009B009A5823005E33C4
:1046E000DD701A70FEBDC046946A0000106A0000BA
:1046F000036910B51A00FC32D2680400002A0AD0FF
:10470000A322D20099581430C9B2FFF754FE0022F8
:104710002369FC33DA6010BD10B50248FFF7E8FFEB
:1047200010BDC0465C0B0020162307B50222009383
:104730000249013B0248FFF7AFFF07BD00200040E0
:104740005C0B00207047000010B500F047F8FFF741
:10475000F9FF012000F024F8FFF792F9FFF7A2F922
:10476000024B002BFAD000E000BFF7E7000000008A
:10477000084A0949094B10B51B688858FA22190ADA
:104780001B0618439200002300F0DCF94904C00B1B
:10479000084310BD0405000000100140C00B0020BC
:1047A00070B5041E09D0FFF7E3FF050000F014F810
:1047B000FFF7DEFF401B8442F8D870BD0022044B97
:1047C0009A60044A13680133DBB213607047C04635
:1047D000FC100140C00B002070470000C421114AAA
:1047E00089005058104B0340C0200002034353502F
:1047F000802391399B02FF39535013608023A322F9
:104800000021DB05D20099500122A1209A60074BBC
:10481000C0001950C1200231800019504030195099
:104820001A60704700E100E0FF00FFFF0010014048
:1048300002B4714649084900095C49008E4402BC33
:104840007047C04603B47146490840004900095A00
:1048500049008E4403BC7047002243088B4274D346
:1048600003098B425FD3030A8B4244D3030B8B4271
:1048700028D3030C8B420DD3FF22090212BA030C7A
:104880008B4202D31212090265D0030B8B4219D35B
:1048900000E0090AC30B8B4201D3CB03C01A52417B
:1048A000830B8B4201D38B03C01A5241430B8B42C3
:1048B00001D34B03C01A5241030B8B4201D30B03AC
:1048C000C01A5241C30A8B4201D3CB02C01A5241D3
:1048D000830A8B4201D38B02C01A5241430A8B4296
:1048E00001D34B02C01A5241030A8B4201D30B027F
:1048F000C01A5241CDD2C3098B4201D3CB01C01A99
:10490000524183098B4201D38B01C01A52414309A2
:104910008B4201D34B01C01A524103098B4201D390
:104920000B01C01A5241C3088B4201D3CB00C01AFD
:10493000524183088B4201D38B00C01A5241430875
:104940008B4201D34B00C01A5241411A00D201469A
:10495000524110467047FFE701B5002000F0F0F823
:1049600002BDC0460029F7D076E7704703460B43E7
:104970007FD4002243088B4274D303098B425FD358
:10498000030A8B4244D3030B8B4228D3030C8B4284
:104990000DD3FF22090212BA030C8B4202D312126A
:1049A000090265D0030B8B4219D300E0090AC30B3F
:1049B0008B4201D3CB03C01A5241830B8B4201D3EC
:1049C0008B03C01A5241430B8B4201D34B03C01AD5
:1049D0005241030B8B4201D30B03C01A5241C30A4D
:1049E0008B4201D3CB02C01A5241830A8B4201D3BE
:1049F0008B02C01A5241430A8B4201D34B02C01AA8
:104A00005241030A8B4201D30B02C01A5241CDD24C
:104A1000C3098B4201D3CB01C01A524183098B4297
:104A200001D38B01C01A524143098B4201D34B0180
:104A3000C01A524103098B4201D30B01C01A5241E3
:104A4000C3088B4201D3CB00C01A524183088B426A
:104A500001D38B00C01A524143088B4201D34B0053
:104A6000C01A5241411A00D20146524110467047C5
:104A70005DE0CA0F00D04942031000D340425340CA
:104A800000229C4603098B422DD3030A8B4212D38A
:104A9000FC22890112BA030A8B420CD389019211BC
:104AA0008B4208D3890192118B4204D389013AD0F9
:104AB000921100E08909C3098B4201D3CB01C01ACE
:104AC000524183098B4201D38B01C01A52414309E1
:104AD0008B4201D34B01C01A524103098B4201D3CF
:104AE0000B01C01A5241C3088B4201D3CB00C01A3C
:104AF000524183088B4201D38B00C01A5241D9D254
:104B000043088B4201D34B00C01A5241411A00D2D4
:104B10000146634652415B10104601D34042002BD0
:104B200000D54942704763465B1000D3404201B54F
:104B3000002000F005F802BD0029F8D016E7704704
:104B40007047C046F0B54F464646C0B41604360C12
:104B50009946330005042C0C070C150C63437E4367
:104B60006F4365431C0CAD1964199C46A64203D9DA
:104B700080235B02984647446346250CEF191D04C9
:104B80004B464A4343432D0C240464199918C91910
:104B900020000CBC90469946F0BDC0467FB51D0074
:104BA0000A4B06001B68D868002A02D1084C230073
:104BB00001E01300074C0293009133002A000649DC
:104BC000019400F021F800F007FEC046B400002078
:104BD00050650000C46A0000D16A0000084B10B59F
:104BE0000400002B02D0002100E000BF054B186834
:104BF000836A002B00D09847200001F0D7FAC04606
:104C000000000000046B00000EB403B5010003AB0C
:104C1000044804CB0068019300F016F902B008BC08
:104C200003B01847B40000200E4B70B500251E00DD
:104C30000D4CE41AA410A54204D0AB00F3589847D9
:104C40000135F8E701F0B4FA084B00251E00084CC6
:104C5000E41AA410A54204D0AB00F35898470135DC
:104C6000F8E770BDBC000020BC000020BC000020A4
:104C7000CC00002010B5034B0100186800F066F866
:104C800010BDC046B400002010B5034B01001868E9
:104C900000F016F810BDC046B4000020002310B587
:104CA0009A4203D0CC5CC4540133F9E710BD030031
:104CB0008218934202D019700133FAE7704700005E
:104CC00030B500293ED004390B68002B00DAC91832
:104CD0001D4A13681400002B02D14B60116031E0B3
:104CE0008B420DD90A688818834203D118685B6823
:104CF00082180A604B60216024E08A4203D81300C6
:104D00005A68002AF9D11D685C198C420BD10968D8
:104D1000691858181960824214D1106852684118F5
:104D200019605A600EE08C4202D90C23036009E03E
:104D300008680C18A24203D1146852682018086051
:104D40004A60596030BDC046C80B0020032370B5CF
:104D5000CD1C9D43083506000C2D01D20C2505E025
:104D6000002D03DA0C230020336040E0A942F9D87B
:104D70001F4B1C681A002100002913D00B685B1B15
:104D80000DD40B2B02D90B60CC181EE08C4202D143
:104D9000636813601AE04B6863600C0016E00C0057
:104DA0004968E9E7134C2368002B03D1300000F079
:104DB00033FB20602900300000F02EFB431CD1D0D3
:104DC0000323C41C9C43A0420AD125602000072273
:104DD0000B30231D9043C31A09D05A42E25006E01B
:104DE000211A300000F018FB431CEED1BAE770BD69
:104DF000C80B0020C40B0020936810B5013B9360E2
:104E0000002B05DA9469A34208DBCBB20A2B05D04C
:104E10001368581C10601970C8B201E000F010FC53
:104E200010BDF8B506000F001400D518AC4208D02C
:104E300021783A003000FFF7DFFF0134431CF5D141
:104E400000E00020F8BD0000F0B59FB006000F00A4
:104E500002920593002804D08369002B01D100F051
:104E6000B7FD7F4B9F4201D1776808E07D4B9F42A1
:104E700001D1B76803E07C4B9F4200D1F768BB8942
:104E80001B070AD53B69002B07D0002306AD6B61D9
:104E900020336B761033AB763DE03900300000F004
:104EA00027FC0028F1D001204042D6E0059A111DD0
:104EB00012680591002A00DA7FE009920134237814
:104EC0002E2B00D18DE021780322684800F066FE89
:104ED000002807D0654B2A68C01A4023834013433B
:104EE0002B6001342178631C0622614802932976E5
:104EF00000F054FE002800D19DE05E4B002B00D056
:104F000090E00722059B07339343083305936B69B1
:104F1000039A9B186B61029C2378002B04D1029B9F
:104F2000E31A049312D003E0252BF8D00134F3E701
:104F3000049B029A39003000FFF773FF431C00D135
:104F400086E06A69049B944663446B612378002B76
:104F50007ED00122002352426A6002A954325218C4
:104F600001342B60EB60AB601370AB6521780522D8
:104F7000414800F013FE002808D03F4B2A68C01AB1
:104F80000123834013432B600134EFE72B68DA06DB
:104F900004D55322202102A8121811701A0704D533
:104FA00053222B2102A81218117022782A2A00D12C
:104FB0007CE7099B00200A2105E05242EA600222B8
:104FC00013432B607AE72278303A092A04D84B43FE
:104FD00001349B180120F6E7002800D16FE7099300
:104FE0006DE763782A2B0AD1059B02341A1D1B68D2
:104FF0000592002B01DA01235B42079363E700234C
:105000000A201A0001346B6021783039092904D84C
:105010004243013452180123F6E7002B00D152E736
:10502000079250E705AB00933A00144B290030007B
:1050300000E000BF07E005AB00933A000F4B2900EA
:10504000300000F08BF80390039B013300D05EE743
:10505000BB895B0600D526E70B981FB0F0BDC046A4
:105060003C6C00005C6C00007C6C00000E6B00006F
:10507000126B000000000000086B0000234E0000CF
:10508000F7B5170001938A680B6900900C009342F2
:1050900000DA130022003B6043321278002A01D06C
:1050A00001333B6023689B0602D53B6802333B60BB
:1050B000062523681D401ED0230043331B785A1E4B
:1050C0009341226892061CD53020E11843310870C4
:1050D00021005A1C45310978A2184332023311705D
:1050E0000FE022000123193201990098089EB04771
:1050F000431C0ED00135E3683A689B1A9D42F0DBF1
:10510000DAE72200019943320098089DA847431C22
:1051100002D10120404220E006232068E1683A687D
:1051200003400025042B03D18D1AEB43DB171D40F0
:10513000A3682269934201DD9B1AED180027BD4246
:105140000AD0220001231A3201990098089EB04724
:10515000431CDED00137F2E70020FEBDF0B58BB076
:1051600006920A0043320793059004920A7E0C00CF
:10517000109B6E2A00D1ABE011D8632A22D009D847
:10518000002A00D1B5E0582A00D0C5E045310A70A8
:10519000814A4FE0642A1DD0692A1BD0BCE0732AE3
:1051A00000D1AAE009D86F2A29D0702A00D0B3E034
:1051B000202209680A43226037E0752A1FD0782A26
:1051C00033D0A9E00E001A684236111D1960136829
:1051D0003370A4E021681A68080606D4490604D58D
:1051E000111D19600023D55E02E0111D19601568BC
:1051F000002D3BDA2D23049A6D42137036E02168AE
:105200001A68080606D4490604D51568111D1960E8
:10521000ADB202E0111D196015685F4B227E039349
:1052200008276F2A1DD00A271BE02200782145326B
:1052300011705A4A19680392081D226818600D6897
:10524000100602D4500600D5ADB2D30702D52023F4
:105250001A4322601027002D03D1202322689A438D
:1052600022602300002243331A7002E00A274A4BCF
:1052700003936368A360002B09DB04222168914338
:105280002160002D05D1049E002B11D07BE0002D64
:1052900079D0049E28003900FFF764FB039B013E90
:1052A0005B5C280033703900FFF7D6FA051EF1D198
:1052B000082F09D12368DB0706D56368226993426A
:1052C00002DC3023013E3370049B9B1B23612BE0E7
:1052D00009681A68080607D4490605D5111D196022
:1052E0001368A28A1A8004E0111D196013686269AC
:1052F0001A600023049E236116E01A68111D1960CC
:10530000166800216268300000F048FC002801D0D7
:10531000801B6060636803E0260042363270012320
:1053200023610023049A1370079B09AA00932100AC
:10533000069B0598FFF7A4FE431C02D101204042C2
:1053400027E02369320006990598079DA847431C6A
:10535000F4D0236800259B070FD4099BE06898428E
:1053600017DA180015E02200012319320699059872
:10537000079EB047431CE1D00135E368099A9B1AA8
:105380009D42F0DBE9E72600039B42361B78337031
:105390008EE70BB0F0BDC046196B00002A6B000011
:1053A000154B10B51C68A36B002B15D11820FFF707
:1053B00061FC124BA0630380114B01224380114B0F
:1053C0008380114BC380114B038105234381063336
:1053D0008381002302614361A46B0D4A20696169E6
:1053E0000C4BFFF7AFFB01220023801859412061CD
:1053F00061614800400810BDB40000200E33000079
:10540000CDABFFFF341200006DE6FFFFECDEFFFFC7
:105410002D7F954C2DF45158002370B5064C050096
:105420000800236000F0ACFE431C03D12368002B6E
:1054300000D02B6070BDC046E81E00200CB430B513
:10544000164B9DB00C1E1D6804DA8B2301202B60C7
:1054500040421DE0822302A99B008B810023029021
:1054600008619C4200D0631E8B604B6101235B424C
:10547000CB81209A21AB2800019300F037FC431C1C
:1054800001DA8B232B60002C02D00023029A1370C8
:105490001DB030BC08BC02B01847C046B4000020A4
:1054A0000EB410B59DB002A9029008610B48822489
:1054B00088604861012040421FABC881084804CB86
:1054C000A400006801938C8100F010FC0023029A74
:1054D00013701DB010BC08BC03B01847FFFFFF7F5E
:1054E000B4000020031C0A7801311A700133002A2D
:1054F000F9D170470023C25C0133002AFBD1581E4A
:1055000070470000F0B51E00454B87B01B68019244
:10551000029308220B00059003911C7802995D1CF0
:1055200009194878104001D02B00F6E72D2C04D142
:105530009D1C5C780123009304E000902B2C01D18A
:105540005C789D1C002E02D0102E0AD162E0302C17
:105550005ED120222B789343582B54D110266C789F
:105560000235009F31007B1E9F412E4BFF183800F3
:10557000FFF7F8F9380004913100FFF76DF90023C7
:105580000322070094461800029A12195178042247
:10559000114201D0303C07E06246114017D037225B
:1055A000012900D02032A41AA64210DD5A1C0BD0CB
:1055B000B84207D802D1049B9C4203DC704301230C
:1055C000201801E001235B422C780135DCE75A1CEE
:1055D0000BD10098059A431E9841124BC018222304
:1055E0001360019B002B0AD117E0009A002A00D01B
:1055F0004042019A002A10D0039A002B00D06A1E64
:10560000019B1A6009E03024002EAAD10826A8E7E1
:105610000A26A6E7302C9CD0A3E707B0F0BDC04611
:10562000B8000020FFFFFF7F10B513000A00010043
:1056300002480068FFF766FF10BDC046B4000020B6
:10564000F8B505000F001400002804D08369002B72
:1056500001D100F0BDF9234B9C4201D16C6808E0F8
:10566000214B9C4201D1AC6803E0204B9C4200D10D
:10567000EC68A369A360A3891B070AD52369002BE3
:1056800007D023682269FEB2981A636998420FDB3B
:1056900008E02100280000F02BF80028F1D00120BC
:1056A00040421DE02100280000F024F90028F6D136
:1056B000A3680130013BA36023685A1C22601F705D
:1056C0006369984205D0A3893000DB0708D50A2E0C
:1056D00006D12100280000F00DF90028DFD13000AC
:1056E000F8BDC0463C6C00005C6C00007C6C0000A7
:1056F000354B70B51D6806000C00002D05D0AB6958
:10570000002B02D1280000F063F9304B9C4201D1FC
:105710006C6808E02E4B9C4201D1AC6803E02D4B35
:105720009C4200D1EC68A3899AB2110723D4D10618
:1057300007D409220120326037321343A38140424B
:1057400040E0530713D5616B002908D02300443390
:10575000994202D03000FFF7B3FA0023636324229A
:10576000A3899343A38100236360236923600822F4
:10577000A3891343A3812369002B0BD1A023A28902
:105780009B00134080229200934203D021003000FE
:1057900000F0B2F90123A289134005D00023A360D1
:1057A00063695B42A36103E0910700D46369A3606E
:1057B00000202369834205D1130603D540231A43F1
:1057C000A281013870BDC046B40000203C6C0000CE
:1057D0005C6C00007C6C000010B5062000F0AEFB95
:1057E000012000F0E3FC0000F7B58A8905000C00F9
:1057F00013075AD44B68002B02DC0B6C002B19DD0D
:10580000E76A002F16D000232E682B6080235B01EF
:105810001A4001D0606D14E00123216A2800B847C6
:10582000431C0ED12B68002B0BD01D2B01D0162B47
:1058300002D12E6000205AE04022A3891343A381A5
:1058400055E0A3895B0706D56368C01A636B002B1C
:1058500001D0236CC01A00230200216A2800E76AE5
:10586000B847A389421C06D129681D293AD8204A85
:10587000CA40D20736D50022626022692260DB046A
:1058800005D5431C02D12B68002B00D16065616BEC
:105890002E600029CED023004433994202D0280044
:1058A000FFF70EFA0020606321E00F69002FC1D0DE
:1058B0000B680F60DB1B01930023920700D14B693B
:1058C000A36003E0019B3F181B1A0193019B002B6F
:1058D000B0DD019B3A00216A2800A66AB047002883
:1058E000F0DCA389402201201343A3814042FEBD86
:1058F000010040200B6970B505000C00002B01D1A0
:1059000000201CE0002804D08369002B01D100F0A6
:105910005FF80B4B9C4201D16C6808E0094B9C423C
:1059200001D1AC6803E0084B9C4200D1EC680C222A
:10593000A35E002BE4D021002800FFF755FF70BDC7
:105940003C6C00005C6C00007C6C000010B50249EF
:1059500000F0B0F810BDC046F5580000002310B5A7
:10596000040003604360836081814366C2810361F8
:1059700043618361190008225C30FFF798F9054BF9
:1059800024626362044BA362044BE362044B23630F
:1059900010BDC0467D5F0000A55F0000DD5F000018
:1059A0000960000070B568254B1E5D430E0029009C
:1059B0007431FFF7CBF9041E08D000212A000160E2
:1059C00046600C30A0606832FFF771F9200070BDAE
:1059D000836913B50400002B28D18364C364036575
:1059E000134B144A1B6882620193984201D1012330
:1059F0008361200000F020F86060200000F01CF8B7
:105A0000A060200000F018F80022E0600421606827
:105A1000FFF7A4FF01220921A068FFF79FFF0222E0
:105A20001221E068FFF79AFF0123A36113BDC0466E
:105A3000046B00004D590000F8B51D4B06001D68B1
:105A4000AB69002B02D12800FFF7C2FF4835AC68D4
:105A50006B68013B05D40C22A75E002F10D0683480
:105A6000F7E72B68002B01D02D68F0E70421300008
:105A7000FFF798FF28600028F6D10C23336016E06A
:105A8000012320005B42E3810233A3816766276024
:105A9000A760676027616761A7615C3008223900F1
:105AA000FFF705F920006763A763A764E764F8BD03
:105AB000046B0000F7B5040007000026019148348C
:105AC000002C16D06368A5680093009B013B0093EF
:105AD0000DD4AB89012B08D90E22AB5E013304D063
:105AE00029003800019B984706436835EDE7246894
:105AF000E6E73000FEBD0000F0B58B8991B00600EE
:105B00000C009B0726D40E23C95E002904DA8023EB
:105B1000A5891D4010D10CE001AA00F0A1FA0028CF
:105B2000F5DBF023029D1B021D401A4BED186B4262
:105B30005D418027FF0001E000254027390030004B
:105B4000FFF704F900280CD1A3899A051FD402227B
:105B50001343A3812300473323602361012363613F
:105B600015E080220C4BB362A38920601343A3810C
:105B700020616761002D0AD00E23E15E300000F045
:105B800081FA002803D00122A3891343A38111B015
:105B9000F0BDC04600E0FFFF4D590000C9B28218B9
:105BA000904204D003788B4202D00130F8E7002005
:105BB000704710B5884202D98B18984201D3002350
:105BC00005E09B1A013A08D3995C8154FAE79342A5
:105BD00003D0CC5CC4540133F9E710BDF8B506001E
:105BE0000C001500002904D11100FFF7AFF80400E4
:105BF00018E0002A03D1FFF763F82C0012E000F050
:105C000067FA85420ED929003000FFF79FF8071E7A
:105C100007D021002A00FFF741F821003000FFF7EC
:105C20004FF83C002000F8BDF0B58E6885B0070045
:105C30000C00039201939E4243D890238A89DB0093
:105C40001A423ED003250969236801985B1A029322
:105C500063695D43EB0F5D19029B6D1001331B18E7
:105C6000AB4200D91D00530510D529003800FFF7BD
:105C70006DF8061E14D0029A2169FFF70FF8A28969
:105C8000194B134080221343A38112E02A003800ED
:105C9000FFF7A4FF061E0CD121693800FFF710F8AA
:105CA0000C23402201203B60A38940421343A3817F
:105CB00017E0029B2661F61826606561019EED1AC9
:105CC000A560019BB34200D21E00320003992068F8
:105CD000FFF76FFF0020A3689B1BA36023689E193A
:105CE000266005B0F0BDC0467FFBFFFFF0B59FB05A
:105CF000029005938B890F0016001B0610D50B69C7
:105D0000002B0DD14021FFF721F8386038610028C1
:105D100004D10C23029A01381360D8E040237B6140
:105D2000002306AD6B6120336B761033AB76340005
:105D30002378002B03D1A31B049312D003E0252B5F
:105D4000F9D00134F4E7A31B320039000298FFF7C1
:105D50006BFF431C00D1B4E06A69049B9446634422
:105D60006B612378002B00D1ABE00122002352426B
:105D70006A6002A95432521801342B60EB60AB60A8
:105D80001370AB65534E217805223000FFF706FFF4
:105D9000002807D00123801B83402A680134134365
:105DA0002B60EFE72B68DA0604D55322202102A8E6
:105DB000121811701A0704D553222B2102A81218A9
:105DC000117022782A2A03D0099B00200A210EE0B4
:105DD000059A111D12680591002A01DB099204E061
:105DE0005242EA60022213432B6001340BE0227816
:105DF000303A092A04D84B4301349B180120F6E7B6
:105E0000002800D0099323782E2B1ED163782A2BEB
:105E10000AD1059B02341A1D1B680592002B01DA7A
:105E200001235B42079310E000230A201A0001348B
:105E30006B6021783039092904D842430134521863
:105E40000123F6E7002B00D00792234E217803228E
:105E50003000FFF7A3FE002806D04023801B8340BC
:105E60002A68013413432B60217806221B48661CE4
:105E70002976FFF793FE002812D0194B002B06D18C
:105E80000722059B073393430833059314E005ABC2
:105E900000933A00134B2900029800E000BF07E08E
:105EA00005AB00933A000F4B29000298FFF756F913
:105EB0000390039B013304D06B69039A9B186B61B9
:105EC00035E7BB890B985B0601D5012040421FB026
:105ED000F0BDC046086B00000E6B0000126B0000A6
:105EE00000000000295C000070B504000D1E1F2D8D
:105EF00004D916230360012040421EE0426C002AB0
:105F000004D08B00D2181368002B08D1200000F0B9
:105F100031F82A000100200000F01AF80DE00020FE
:105F2000012B0AD0591C03D117332360013004E040
:105F30000024280014609847200070BD10B5034B62
:105F400001001868FFF7D0FF10BDC046B400002064
:105F5000002370B5064C050008001100236000F016
:105F6000F7F8431C03D12368002B00D02B6070BDD1
:105F7000E81E002010B500F0DBF810BD70B50C0075
:105F80000E25495F00F0B0F8002803DB636D1B1895
:105F9000636503E0A289024B1340A38170BDC04634
:105FA000FFEFFFFFF8B51F008B8905000C001600FE
:105FB000DB0505D50E23C95E0022022300F074F82C
:105FC000A289054B28001340A38132000E23E15E15
:105FD0003B0000F01FF8F8BDFFEFFFFF70B50C00AD
:105FE0000E25495F00F060F8A389421C03D1054AE1
:105FF0001340A38104E0802252011343A381606512
:1060000070BDC046FFEFFFFF10B50E23C95E00F064
:1060100015F810BD70B50500080011000022064CEF
:1060200022601A0000F0BAF8431C03D12368002B49
:1060300000D02B6070BDC046E81E0020002370B564
:10604000064C05000800236000F062F8431C03D1F1
:106050002368002B00D02B6070BDC046E81E0020D6
:10606000002370B5064C050008001100236000F005
:1060700057F8431C03D12368002B00D02B6070BD60
:10608000E81E0020002370B5064C050008002360C0
:1060900000F056F8431C03D12368002B00D02B607E
:1060A00070BDC046E81E002070B505000800110054
:1060B0000022064C22601A0000F052F8431C03D163
:1060C0002368002B00D02B6070BDC046E81E002066
:1060D0000B1F1A68101F002A04DA891804390B688C
:1060E000D01804387047000070B505000800110092
:1060F0000022064C22601A0000F03AF8431C03D13B
:106100002368002B00D02B6070BDC046E81E002025
:1061100058220120014B40421A607047E81E0020BF
:1061200058220120014B40421A607047E81E0020AF
:1061300058220120014B40421A607047E81E00209F
:106140005822024B00201A607047C046E81E00200B
:1061500058220120014B40421A607047E81E00207F
:1061600058220120014B40421A607047E81E00206F
:1061700058220120014B40421A607047E81E00205F
:10618000044A1368002B03D01818106018007047D9
:10619000014BF9E7CC0B0020F01E00205822012013
:1061A000014B40421A607047E81E0020FEE7C046DF
:1061B000F8B5C046F8BC08BC9E467047F8B5C04666
:1061C000F8BC08BC9E467047AE06000040060000C2
:1061D000BE060000F4060000300700006A07000059
:1061E000A6070000D20700001008000056080000B3
:1061F000B2080000F808000066090000B4090000B9
:10620000E00900001A0A0000640A00008C0A00007D
:10621000C40A0000FC0A0000380B0000BE0B00009E
:10622000860C0000F40C0000300D0000720D000020
:10623000940D00009C0D00007C0E0000AE060000D6
:10624000AE060000AE060000AE060000AE0600007E
:10625000AE060000C80E0000120F0000600F000024
:10626000E60F000082100000D01000001A1100009C
:1062700060110000AC110000F81100004412000091
:1062800090120000DC1200001A13000086130000B8
:10629000B61300000C14000058140000A4140000F1
:1062A000DE1400002A150000AE060000AE06000055
:1062B000AE060000AE06000076150000A615000030
:1062C000D615000002160000321600005E1600000F
:1062D000AE060000AE060000AE060000AE060000EE
:1062E0008E160000D616000022170000521700007C
:1062F0007E170000C4170000AE060000AE060000C6
:10630000AE060000AE0600000418000034180000BD
:106310006418000094180000C0180000F018000075
:106320001C1900004619000070190000A019000097
:10633000D0190000FC190000281A0000581A0000AB
:10634000841A0000AE060000AE060000AE06000093
:10635000AE060000AE060000B41A0000E01A00000D
:106360000C1B0000381B0000741B0000A41B000065
:10637000D41B0000041C0000341C0000601C000042
:106380008E1C0000BE1C0000EC1C00002C1D000038
:106390005C1D0000AE060000AE060000AE06000068
:1063A000AE060000AE060000AE060000AE0600001D
:1063B000AE060000AE060000AE060000AE0600000D
:1063C000AE060000AE06000066616C736500747274
:1063D0007565006C697374206F662025642069748C
:1063E000656D73006F626A656374206F6620636C0D
:1063F0006173733A20256400537461636B20756E7A
:10640000646572666C6F77000D0A564D2050616EA0
:1064100069633A2025730D0A00496E7375666669D3
:106420006369656E74206D656D6F727920666F7239
:10643000204D6963726F426C6F636B73206F626A89
:10644000656374206865617000496E73756666697E
:106450006369656E74206D656D6F727920666F7209
:10646000204D6963726F426C6F636B73207374614C
:10647000636B00626164206F626A6563742061749B
:1064800020256C640A0025783A20256420776F72F5
:1064900064732C20636C61737349442025640A0083
:1064A0004865616465723A2025780A0009307825CC
:1064B000782C0A0025642025642025642025640AA0
:1064C00000426164207265636F726420666F756E4E
:1064D0006420647572696E6720696E697469616CA5
:1064E000697A6174696F6E210A004E6F7420656E5F
:1064F0006F75676820726F6F6D206576656E2061BD
:106500006674657220636F6D70616374696F6E0A83
:1065100000526573746F72696E672025642073631F
:1065200072697074732E2E2E0053746172746564D8
:10653000002D2D2D2D2D0A00506572736973746521
:106540006E74204D656D6F727920546573740A0AFC
:10655000000A496E697469616C697A696E67204DD9
:10656000656D6F72790A004D656D6F727920696E85
:1065700074697469616C697A65643B2077726974C7
:10658000696E67207265636F7264732E2E2E0A0027
:106590005265636F7264206174206F666673657400
:1065A0002025643A20256420256420256420256464
:1065B0002028256420776F726473290A0046696E6B
:1065C000616C3A2063757272656E74202564207563
:1065D00073656420256420633020256420633120A6
:1065E00025640A004E6F2066726565207461736BC6
:1065F00020656E747269657300416C6C2074617300
:106600006B732073746F7070656400763034320081
:106610002025732025730057656C636F6D652074AA
:106620006F204D6963726F426C6F636B7321001A48
:106630001B1C03040607090A1718190000000000B4
:106640000100000002000000030000000400000040
:106650000500000006000000070000000800000020
:10666000090000000A0000000B0000000C00000000
:106670000D0000000E0000000F00000010000000E0
:1066800012000000140000001600000018000000B6
:106690001A0000001C0000001E0000002000000086
:1066A0002300000026000000290000002C0000004C
:1066B0002F00000032000000360000003A00000009
:1066C0003E00000042000000460000004B000000B9
:1066D00050000000550000005A000000610000005A
:1066E000680000006F000000760000007D000000E0
:1066F000840000008B000000920000009900000060
:10670000A0000000A7000000AE000000B5000000DF
:10671000BC000000C3000000CA000000D10000005F
:10672000D8000000DF000000E6000000ED000000DF
:10673000F4000000FB000000FF000000000000006B
:106740000008080800080A4A4000000A5FEA5FEAF9
:106750000ED92ED36E19324489330C924C924D08C7
:106760000800000004880808040804848488000ADB
:10677000448A4000048EC480000000048800000E9B
:10678000C000000000080001224488100C92525200
:106790004C048C84848E1C824C901E1EC244924CED
:1067A00006CA525FE21FF01EC13E02448ED12E1F68
:1067B000E24488100ED12ED12E0ED12EC4880008AE
:1067C00000080000048004880244880482000EC08F
:1067D0000EC008048244880ED126C0040ED135B301
:1067E0006C0C925ED2521C925C925C0ED010100E19
:1067F0001C9252525C1ED01C901E1ED01C90100E7B
:10680000D013712E12525ED2521C8808081C1FE24F
:1068100042524C1254981492101010101E113B75D5
:10682000B131113935B3710C9252524C1C925C90BB
:10683000100C92524C861C925C92510ED00C825CD1
:106840001FE4848484125252524C1131312A441173
:106850003135BB7112524C9252112A4484841EC4A9
:1068600088101E0EC808080E10080482410EC2428D
:10687000424E048A400000000000001F080480000F
:1068800000000ED2524F10101C925C000ED0100E61
:1068900002424ED24E0C925C900E06C81C88080E26
:1068A000D24EC24C10101C92520800080808024038
:1068B00002424C10149814920808080806001B7530
:1068C000B131001C925252000C92524C001C925C4E
:1068D00090000ED24EC2000ED010100006C80498D0
:1068E00008080EC807001252524F0011312A440006
:1068F000113135BB00124C8C9200112A4498001EB5
:10690000C4881E06C48C8486080808080818080C69
:10691000881800000C83606D6963726F3A62697455
:106920000000000000000000010000000200000064
:1069300003000000040000000A0000005350494317
:106940006C6173733A3A535049436C617373284EC8
:1069500052465F5350495F547970652A2C207569FF
:106960006E74385F742C2075696E74385F742C20D7
:1069700075696E74385F742900705F7370692021C7
:106980003D204E554C4C002F55736572732F6A6F26
:10699000686E6D616C6F6E65792F4C6962726172A1
:1069A000792F41726475696E6F31352F7061636B39
:1069B000616765732F73616E646565706D6973746B
:1069C00072792F68617264776172652F6E524635F5
:1069D0002F302E342E302F6C6962726172696573AC
:1069E0002F5350492F5350492E6370700000000000
:1069F0000000000000000000533C0000193C0000B3
:106A00003F3C0000493C0000793C00003D3C000058
:106A1000030000000200000001000000040000006C
:106A200005000000110000000C0000000B00000039
:106A3000120000000A000000060000001A0000001A
:106A400014000000170000001600000015000000F0
:106A500010000000FFFFFFFFFFFFFFFF000000002E
:106A60001E000000190000001800000007000000D0
:106A700008000000090000000D0000000E000000EA
:106A80000F0000001C0000001B0000001D000000A3
:106A9000130000000000000000000000354400006A
:106AA00055430000A5440000B9440000AF44000075
:106AB0003344000027440000C54400005144000056
:106AC000234400002C2066756E6374696F6E3A2053
:106AD00000617373657274696F6E202225732220C2
:106AE0006661696C65643A2066696C65202225736D
:106AF000222C206C696E65202564257325730A009D
:106B00004300000054000020232D302B2000686C2F
:106B10004C006566674546470030313233343536C0
:106B200037383941424344454600303132333435F9
:106B300036373839616263646566000020202020A2
:106B4000202020202028282828282020202020201D
:106B500020202020202020202020202088101010FD
:106B60001010101010101010101010100404040455
:106B700004040404040410101010101010414141CA
:106B80004141410101010101010101010101010135
:106B900001010101010101101010101010424242C8
:106BA0004242420202020202020202020202020205
:106BB0000202020202020210101010200000000067
:106BC00000000000000000000000000000000000C5
:106BD00000000000000000000000000000000000B5
:106BE00000000000000000000000000000000000A5
:106BF0000000000000000000000000000000000095
:106C00000000000000000000000000000000000084
:106C10000000000000000000000000000000000074
:106C20000000000000000000000000000000000064
:106C30000000000000000000000000000000000054
:106C40000000000000000000000000000000000044
:106C50000000000000000000000000000000000034
:106C60000000000000000000000000000000000024
:106C70000000000000000000000000000000000014
:106C80000000000000000000000000000000000004
:106C900000000000000000000000000000000000F4
:086CA000D494FF7F0100000005
:106CA800FFFFFFFF180000000300000002000000C3
:106CB800080000000A000000FFFFFFFF00000000BE
:106CC800010000000000020001000000FFFFFFFFBC
:106CD80000000000020000000000040002000000A4
:106CE800FFFFFFFF00000000030000000000080095
:106CF80003000000000000003C6C00005C6C000019
:106D08007C6C000000000000000000000000000093
:106D180000000000006B0000000000000000000000
:106D2800000000000000000000000000000000005B
:106D3800000000000000000000000000000000004B
:106D4800000000000000000000000000000000003B
:106D580000000000540000203B6B000039010000D7
:106D6800E93B0000CD3E0000294700000D0100006E
:046D78000000000017
:0400000300003EE5D6
:00000001FF
